:1074B300758400852ED2852FD3E4F52FF52E303831
:1074C30010E50D852DF0A4252EF52EE5F0352FF5CD
:1074D3002F229074EF303E031274DF22E50E251B3A
:1074E300F50EE51F351AF51F93F50D227F8285886A
:1074F3008C8F9295989B9EA1A4A7AAADB0B3B6B961
:10750300BBBEC1C3C6C9CBCED0D3D5D7D9DCDEE091
:10751300E2E4E6E7E9EBEDEEF0F1F2F4F5F6F7F885
:10752300F9FAFBFCFCFDFDFEFEFEFEFEFEFEFEFE8A
:10753300FEFDFDFCFCFBFAFAF9F8F7F6F4F3F2F0C2
:10754300EFEDECEAE8E7E5E3E1DFDDDBD8D6D4D124
:10755300CFCDCAC8C5C2C0BDBAB7B4B2AFACA9A675
:10756300A3A09D9A9794908D8A8784817E7A77745D
:10757300716E6B6865625F5C595653504D4A474460
:10758300423F3C393734322F2D2A282624211F1D10
:107593001B1918161412110F0E0C0B0A08070605F7
:1075A30004040302020101000000000000000000C7
:1075B3000001010202030405060708090A0B0D0E68
:1075C3001011131516181A1C1E20222427292B2EDE
:1075D300303335383A3D404245484B4E5154565965
:0C75E3005C606366696C6F7275787B7F7A
:107CE400D2F4C2F5C2F675840F85F0C8127A3074E6
:107CF40003127D33127A207403127D33127A0F1229
:107D04007A0F7403127D33127A0F7402127D3312C8
:107D14007A0F7428127D9F7406127D9F740E127D53
:107D24009F7401127D9F127A207480127D9F22C05D
:107D340000A2E092F3A2E192F2A2E292F1A2E39213
:107D4400F0D2F475840F85F0C8C2F47830D8FE857B
:107D5400F0C87830D8FED00022C00075840FA2E4A9
:107D640092F3A2E592F2A2E692F1A2E792F0D2F4A3
:107D740085F0C8C2F47830D8FE85F0C87830D8FED3
:107D8400D00022EF75840FD2F5C2F685F0C8127DBB
:107D94005D127A0F127D33127A0F2275840FC2F5A9
:107DA400C2F685F0C8127D5D127A0F127D33127A05
:107DB4000F22EF14A2E492E6C2E4D2E7127D9F22DE
:107DC400740F127D9F22740D127D9F227F01127DFC
:107DD400B678107F20127D87D8F9227F11127DB6E4
:0A7DE40078107F20127D87D8F92265
:10737600C293758400D2C2C2C6D2C6C2C4D2C5C226
:10738600C330C3FD74A0F5C2C2C5C2C330C3FD8EEF
:10739600C2C2C330C3FD8FC2C2C330C3FD8DC2C2D9
:1073A600C330C3FDD2C4C2C320C4FD127A20D29317
:1073B60022758400C2C3D2C530C3FD74A0F5C2C213
:1073C600C5C2C330C3FD8EC2C2C330C3FD8FC2C2A5
:1073D600C330C3FDC2C4D2C5C2C330C3FD74A1F558
:1073E600C2C2C5C2C330C3FDC2C2C2C330C3FD855B
:1073F600C207D2C4C2C320C4FD22D2C2C2C6D2C6EC
:10740600D2C4C2C320C4FD22C293758400D2C2C2B4
:10741600C6D2C6C2C4D2C5C2C330C3FD74A0F5C2AB
:10742600C2C5C2C330C3FD8EC2C2C330C3FD8FC244
:10743600C2C330C3FD8C838D827B80E0A3F5C2C2BC
:10744600C330C3FDDBF5D2C4C2C320C4FD127A200B
:10745600D29322758400C2C3D2C530C3FD74A0F591
:10746600C2C2C5C2C330C3FD8EC2C2C330C3FD8F04
:10747600C2C2C330C3FDC2C4D2C5C2C330C3FD74C9
:10748600A1F5C2C2C5C2C330C3FD8C838D82C2C3FF
:1074960030C3FDE5C2F0A31BBB01F3C2C2C2C330B9
:0D74A600C3FDE5C2F0D2C4C2C320C4FD2264
:030003000259C2DD
:01000B0032C2
:0300130002772A47
:1066180075FF0775FFDE75FFAD75840F75E10775AA
:10662800E21475E34475840F75A43575A50975A63C
:10663800BB75A7FF759CFF759D00759EF0759FF84B
:1066480075D8FF75E8FF75F80F75AD0F758401757E
:10665800893075888F75840275893075888F75843F
:106668000F758A80758C67780874FF000000000039
:1066780000000000000000D5E0F1D8EDE58C30E71F
:10668800FB759701758A0043890475840075B710F6
:1066980075840F438901758D02758F01758E047499
:1066A80080D5E0FD438902E58930E4FB75970275E2
:1066B800840075D10775840075BB0175BA0075BC77
:1066C800F075C70075C60075C5FF75C4FF75E8008D
:1066D80075840275BB0475BA0075BCF175C6007582
:1066E800C4FF75E88075840075D48475840175D4F9
:1066F80084758400C2F8759A47759D1A75F80175F6
:10670800870075840075B90075A9007591007598A2
:106718005075840175989075840075C04075C300E4
:1067280075CFC9758400758E1075892175880575B2
:106738008400758A00758BE0758CF4758DE043884C
:106748004075840075C90075CA0075CB0075CC000A
:1067580075CD0075840175C91875CA8075CBFB7530
:10676800CDFB75CC80D2CA75840275C91875CAA6C6
:1067780075CBAF75CDAF75CCA6D2CA75840075EF51
:106788000275A8AC75B83D75E6B075E71D75F600DD
:1067980075F741789D760A769E780A789F76067511
:0767A800A8959000007F009E
:1067AF007E20E4F0A3DFFCDEFA789D760A789E76F1
:0E67BF000A789F7606D29375E8FF12740022C6
:1079890075840FD2FD2275840FC2FD22E490FC009C
:10799900732275840FD2EA2275840FC2EA22758494
:1079A9000FA2EC2275840FD2FC2275840FC2FC222F
:1079B90075840FC2FF2275840FD2FF2275840FA22E
:1079C900FA2275840FA2F92275840FA2DD22A292F0
:1079D9002275840FA2DA2275840FA2DB2275840F27
:1079E900A2D82275840FA2D922000000000000004D
:1079F900000000000000000000000000000000007E
:107A0900000000000022C000C001790878B4D8FE47
:107A1900D9FAD001D00022C000C0E078997605E6F5
:107A290070FDD0E0D00022C000C0E07899760FE662
:107A390070FDD0E0D00022C000C0E078997664E6FD
:107A490070FDD0E0D00022EF75F0648424309000FE
:107A590054F0E5F0A375F00A842430F0A3E5F0248E
:107A690030F022EF75F064842430900054F0E5F092
:097A7900A375F00A842430F0A387
:107A8200E5F02430F0900054E0B4300B7420F0A301
:107A9200E0B430037420F02275F06484F6E5F00857
:107AA20075F00A84F608A6F00822850607222285C8
:037AB200050622A4
:101A1A00C0D0C000C001C083C082C0E0C0F0C0070F
:101A2A00A291304F01B37825E233F208E233F2088B
:101A3A00E233F208E233F208E233F208E233F20860
:101A4A00E233F208E233F208E233F208E233F20850
:101A5A00E233F208E233F208E233F208E233F20840
:101A6A00E233F208E233F208E233F208E233F20830
:101A7A00E233F208E233F208E233F208E233F20820
:101A8A00E233F208E233F208E233F208E233F20810
:101A9A00E233F208E233F208E233F208E233F20800
:101AAA00E233F208E233F208E233F208E233F208F0
:011ABA00E249
:101ABB0033F208E233F208E233F208E233F208E2DF
:101ACB0033F208E233F2305B35901EE7784CE218C4
:101ADB00203C03936028E218937023E21893601E56
:101AEB00E218937019E218936014E21893600FE2F6
:101AFB001893700AE218937005E218936003021CA6
:101B0B00C0754000E2189313924750037540387527
:101B1B002200E21893139214500363401CE21893B3
:101B2B00139213500363400EE21893139212500357
:101B3B00634046E218931392115003634023E2185B
:101B4B00931392108522415003634051752200E29A
:101B5B0018931392145003634068E2189313921373
:101B6B005003634075E21893139212500363407A4B
:101B7B00E21893139211500363403DE218931392B2
:101B8B0010852242500363401F752200E218931305
:101B9B009217500363404FE218931392165003634E
:101BAB004026E218931392155003634052E21893A8
:101BBB001392145003634029E218931392135003AA
:101BCB00634015E21893139212500363400BE21813
:101BDB00931392115003634045E2189313921085AF
:101BEB0022435003634062E2189313921450036331
:101BFB004031E218931392135003634019E2189388
:101C0B00139212500363400DE21893139211500379
:101C1B00634007E2189313921085224450036340EC
:101C2B0043752200E21893139216E2189313921540
:101C3B00E21893139214E21893139213E21893136E
:101C4B009212E21893139211E218931392108522B9
:101C5B0045C24CE54565406035D24C23F89024389D
:101C6B0093F9902437E8936025B40104B247801EA2
:0E1C7B00B40205E862418016B40305E8624237
:101C8900800EB40405E862438006B4052AE862447C
:101C9900A247924890004DE541F090004EE542F090
:101CA90090004FE543F0900050E544F0304B06D2E8
:101CB9004AC24B8002D24B121CD4D007D0F0D0E0DC
:101CC900D082D083D001D000D0D022C0D0C000C0F3
:101CD900E0303F4EE552B40833A242B392B3787D67
:101CE900E66036167882E6A2E7304401B392429262
:101CF900B2A2E7787EE633F6787FE633F67880E6B7
:101D090033F67881E633F67882E633F6D5520375F1
:101D19005208D0E0D000D0D022C257D0E0D000D0B5
:101D2900D022D0E0D000D0D022C0D0C000C001C0A5
:101D390083C082C0E0C0F0A291204E01B3780DE2C9
:101D490013F208E213F208E213F208E213F208E2CE
:101D590013F208E213F208E213F208E213F208E2BE
:0D1D690013F208E213F208E213F208E2138D
:101D7600F208E213F208E213F208E213F208E213A1
:101D8600F208E213F208E213F208E213F208E21391
:101D9600F208E213F208E213F208E213F2901EE7E9
:101DA600780DE2089313920FE2089313920EE2085D
:101DB6009313920DE2089313920CE2089313920B7D
:101DC600E2089313920AE20893139209E208931326
:101DD6009208852146E2089313920FE20893139224
:101DE6000EE2089313920DE2089313920CE2089305
:101DF60013920BE2089313920AE20893139209E2F4
:101E06000893139208852147E2089313920FE2087C
:101E16009313920EE2089313920DE2089313920C19
:011E2600E2D9
:101E2700089313920BE2089313920AE20893139212
:101E370009C208852148305B3DE546902237854732
:101E470021300E02058393602D14F875F003A490DA
:101E570020E82582F582E5F03583F583E493F9A33D
:101E6700E493901FE7654893C965479329B4010038
:101E770050048834D241121E8FD0F0D0E0D082D0E7
:101E870083D001D000D0D022303D27C392B27883CF
:101E970016E6701E76087886E6A2E1304501B39211
:101EA700B3A2E17884E613F67885E613F67886E63A
:101EB70013F622EF9020E775F003A42582F582E55B
:101EC7008335F0F583C23D7400937884F6740193EB
:101ED7007885F67402937886F6C23FC23ED23D22D9
:101EE70000000000000000000000000000000000EB
:101EF70000000000000000000000000000000001DA
:101F070000000000000000000000000000000001C9
:101F170000000000000000010000000100010101B5
:101F270000000000000000000000000000000001A9
:101F37000000000000000001000000010001010195
:101F47000000000000000001000000010001010185
:101F5700000000010001010100010101010101016F
:101F67000000000000000000000000000000000169
:101F77000000000000000001000000010001010155
:101F87000000000000000001000000010001010145
:101F9700000000010001010100010101010101012F
:101FA7000000000000000001000000010001010125
:101FB700000000010001010100010101010101010F
:101FC70000000001000101010001010101010101FF
:101FD70000010101010101010101010101010101EB
:101FE70000010102010202030102020302030304CA
:101FF70001020203020303040203030303030405AC
:102007000102020302030304020303040304040599
:10201700020303040304040503040404040505067A
:10202700010202030203030402030303030404057A
:10203700020303040303040503040405040505065A
:102047000203030403040405030404050405050649
:102057000304040504050506040505060506060729
:102067000102020302030304020303040304040539
:102077000203030403040405030404050405050619
:102087000203030403040405030404050405050609
:1020970003040405040505060405050605060607E9
:1020A70002030304030404050304040504050506E9
:1020B70003040405040505060405050605060607C9
:1020C70003040405040505060405050605060607B9
:1020D7000405050605060607050606070607070899
:1020E700FDD00C73700E3CF01AAF101E7F9022ECDF
:1020F7007026D6F02ACBB02CA3F032BEB03417D05E
:102107003CB6D0461FB04E77F050F950526AB056E1
:10211700DE9058BA306ACF3072D270745CD076E8ED
:10212700F0786BD098E5709AF8309CBB50A40F708C
:10213700AA7A70B26730B45DB0B8FCB0C26F50C64F
:1021470055D0CA3D90D489B0DA94F0DCD790E463D7
:10215700B0EA0BF0F43170F8DD310AB571148FF184
:1021670018D1D126EB512AF6112C8B71463F5148D5
:10217700B1F14AACB14CC4F152D9B1546D915A2E58
:10218700F162BD116687916A9AD16CF29172D5514D
:0D2197007819F18C71B192D8D19A32D1AA89
:1021A40047D1B25A91B452F1C67531CC1D71D2A93E
:1021B40051DCD0B1E85E11EA2B11F2EED212F392A7
:1021C400147D3216973226D8B232C5F234F7124A49
:1021D400EA524C9F5254A5D2582B725A7552644FEE
:1021E400D268C1726ADC326C78D2865F128C8372D8
:1021F4009C4EB2A66972AC1C72B433D2CC18F2EA0B
:10220400BB330CCE33141EB32803F32EE51332F87C
:10221400533498735848F36472736845738617B3DC
:10222400947313A63C93B221D3B41B53B829B3C6F9
:1022340041F3D8000000000000000000000000008E
:10224400000000000000000000006A000000000020
:1022540000620D0000000000000000006F00480054
:102264000000000000000000000000000000006CFE
:102274002200000000000000000000000000000038
:10228400005B0000000000000000000000410000AE
:102294001E4759000000260000001D000010000029
:1022A400350000003D006B0043000000000000000A
:1022B4004B0005000000000000003800230000006F
:1022C400000000000000000000004C0000000000BE
:1022D40000000000000000000000000000000032C8
:1022E4000000040000000000000000000012600074
:1022F400370A000000000000000000000000080091
:1023040000611346000000000000254D3400005712
:10231400291100000000000064000000000000001B
:1023240000000000003A4A00002E4F190000001F70
:10233400000000000000630000000000000027000F
:1023440000001B000000000000000B5F3C006E5DFD
:10235400440000006D000000000000000000530075
:1023640000360000283F5E0000000000000000036B
:1023740000003000700000006900406700000000A9
:10238400000055000042000021000000000000157C
:102394000000000000000000000000005C001700C6
:1023A400000020000068020054000E58001C0000C9
:1023B4000000000000005A000000000000002F0090
:1023C40000002B000000002400000066003900001B
:1023D4000000510000000900520000004500000008
:1023E40000000000310000002A0C000000001A0068
:1023F40000000000560000334E0000000000000002
:10240400000000002C1400003B07003E0000000008
:1024140000000000000000001800001600502D0607
:102424000049000000000000000000650F000000EB
:102434000100000000000000000600000006000685
:102444000005020600060006000404060005040256
:102454000806000000060006000600060004080640
:102464000006000600050806000600021006000625
:102474000003010000060006000202060006000434
:1024840040060006000410060006000600060006CA
:1024940000060006000510060006000600060006F9
:1024A40000060001010600060006000600030206FD
:1024B40000060000000600060005010600040202F2
:1024C40004060006000600060006000600060006D4
:1024D400000480060002010420060006000600062F
:1024E40000060006000600060006000600060006B8
:1024F40000060006000600040106000600060006A9
:10250400000600031006000600060006000600068A
:0D2514000006000600060006000600060096
:102521000308060006000600060003040600060074
:0625310006000600060092
:1059C200758400C2CA85CC3885CD3775CC0075CDBB
:1059D20000D2CA10CF02D25A32305A0BC25AE5371D
:1059E200C394364002800122788E798C7B06E7F6DA
:1059F2001819DBFAA63718A638AA38AB37AE02AFA9
:105A020003EEC4035407FEEFC403FF54F84EFEEF47
:105A12005407FF78037989C3E79AFC09E79BFD09DC
:105A220050066304FF6305FFC3EC9EED9F5074D8DC
:105A3200E6789679947C06E7F61819DCFAA603183C
:105A4200A6027991AE02AF03EEC423541FFEEFC447
:105A520023FF54E04EFEEF541FFF7803C3E79AFC86
:105A620009E79BFD0950066304FF6305FFC3EC9E33
:105A7200ED9F502FD8E6788F7A007B007C00790466
:105A8200EA26FA08EB36FB08EC3400FCD9F2EC13F8
:0D5A9200FCEB13FBEA13FAEC13EB13F536F3
:105A9F00EA13F535D23A22303A31C23A125ADB5074
:105AAF002A853C3D853B3C853A3B85393A8507390C
:105ABF00303913E53F6F600EE507B53A0EB53B0B76
:105ACF00B53C08B53D0585073ED23B22905BF6E518
:105ADF003693FF905B2223232582F582E5833400E2
:105AEF00F583125B01400A0F125B0140040F125B3A
:105AFF000122E493F9A3E493FAA3E493FBA3E493C1
:105B0F00FCA3C3E5359AE536995007C3EC9535EB01
:105B1F00953622EA25DD89DD89D324D324CBD2CB58
:105B2F00D2C4DBC4DBBE39BE39B7CAB7CAB18EB176
:105B3F008EAB87AB87A59CA59CA000A0009A969AD8
:105B4F009695D895D891E591E58D858D8588AF8807
:105B5F00AF840C840C7F9A7F9A7B497B49771B77A4
:105B6F001B730F730F6F276F276B576B5767AB67DE
:105B7F00AB642C642C60C660C65D795D795AFE5AA1
:105B8F00FE5970597057E257E25661566154E75407
:105B9F00E7537453745207520750A050A04F404F11
:105BAF00404DE64DE64C934C934B414B4149F549E3
:105BBF00F548B548B547764776463E463E450845D3
:105BCF0008432A432A40E440E43F533F533E3E3EBE
:105BDF003E3C943C943A863A863918391838050079
:105BEF0000000000000000323232323232323232E4
:105BFF003232323232323232323232323232323276
:105C0F003232323232323232323232323232323265
:105C1F003232323232323232323232323232323255
:105C2F00313130302F2E2D2D2D2C2C2B2A29292898
:105C3F0027262525242323222120201F1E1E1D1C3D
:105C4F001C1B1A1A1A1A19191918181817171717B7
:105C5F0016161616151515151414141413131313ED
:105C6F00121212121111111110101010100F0F0F1C
:105C7F000F0F0E0E0E0E0D0D0D0D0C0C0C0C0B0B45
:105C8F000B0B0B0B0A0A0A0A0A0909090909090869
:105C9F000808080808070707070707060606060685
:105CAF00060605050505050504040404040404039C
:105CBF0003030303030302020202020202010101B2
:105CCF0001010101010101010101010000000000BA
:105CDF0000000000000000000000000000000000B5
:075CEF0000000000000000AE
:1070CB00C007C0007F01127DB67F4C127D877F54B5
:1070DB00127D877F52127D877F20127D8720490486
:1070EB007F3080027F31127D877F20127D87900158
:1070FB0091E0784B127AA2784B8607430730127DCA
:10710B0087088607430730127D87750720127D8716
:10711B00900192E0784B127A9A784B8607430730AE
:10712B00127D87088607430730127D870886074341
:10713B000730127D87750720127D87900193E078C9
:10714B004B127AA2784B8607430730127D8708864D
:10715B0007430730127D87750720127D87D000D03B
:10716B000722C007C0007F11127DB67F4C127D87AE
:10717B00750720127D87204D047F3080027F3112EE
:10718B007D877F20127D8790015BE0784B127AA27E
:10719B00784B8607430730127D87088607430730F5
:1071AB00127D87750720127D8790015CE0784B126A
:1071BB007A9A784B8607430730127D8708860743F8
:1071CB000730127D87088607430730127D877507C6
:1071DB0020127D8790015DE0784B127AA2784B8666
:1071EB0007430730127D87088607430730127D87D8
:1071FB00750720127D8790015EE0784B127AA2789A
:10720B004B8607430730127D8708860743073012EA
:07721B007D87D000D007229F
:106E0D00003800512372461765340E5F2D7C4819EA
:106E1D006B3A1C4D3F6E5A0B792812433160540565
:106E2D007726001F3D227A654758756A48570F101F
:106E3D00322D6877554A120D2F301D02203F67788D
:106E4D005A45006245270B694E2C157750321E7C32
:106E5D005B39294B6C0E224067053C5E791B37551B
:106E6D00721052301775593B1C7E472502604C2E0F
:106E7D00096B7B193E5C701235576E0C2B496507FB
:106E8D002042264463012D4F680A33517614385A37
:106E9D007D1F0F6D4A28046641231A785F3D1173DB
:106EAD005436741631537F1D3A58610324466A08CF
:106EBD002F4D5D3F187A56341371482A0D6F4321BB
:106ECD0006644F2D0A68442601635A381F7D5133DD
:106EDD001476660423416D0F284A73113654781ABF
:106EED003D5F1D7F583A16745331086A4D2F03616B
:106EFD004624345671133F5D7A18214364062A489F
:106F0D006F0D690B2C4E620027457C1E395B771582
:106F1D003250402205674B290E6C553710725E3C7E
:106F2D001B793B597E1C305275172E4C6B0925472A
:106F3D00600212705735197B5C3E076542200C6E5E
:106F4D00492B004307440D4E0A49195A1E5D14572B
:106F5D001350317236753C7F3B78286B2F6C25664C
:026F6D0022619F
:10857300788276ACA24DE433FFC4333354C0FE900B
:10858300015DE0FD541F25E04EFE90015BE0FC54CD
:1085930010C4540F4E7881F6EC540FC454F0FE907F
:1085A300015CE0FC54F0C4540F4E7880F6EC540F99
:1085B300C454F0FE90015EE0FC541EC3134E787F5A
:1085C300F6EF3395E0FE740D2FF582746E3EF5835E
:1085D300E493FFED906E0F93FEEF6EFF90015BE06F
:1085E300906E2F936FFF90015CE0906E4F936FFF3F
:1085F300EC906F4F936F787EF690015EE030E0046D
:0B860300E64480F6D257787D762822EE
:10912800758401309914C29920500F900159E0704C
:1091380009D250D29C789776042230983790015AF9
:10914800E06401702DE54975F0058420551124EF80
:10915800F582E43400F583E599F0C298D2552224CB
:1091680004F582E43401F583E599F0C298C255D23A
:059178005622C29822FE
:1080E6007584012098030281AC205213209A0DE575
:1080F600997009D252D253754A0AF549C29822900C
:10810600015AE0FF6401702CE54975F0058420559D
:108116001024EFF582E43400F583E599F0D255801A
:10812600102404F582E43401F583E599F0C255D2B2
:1081360056C29822EFB4021AAB530555E555AA5418
:108146007002055414F9E59912851390015A7403C7
:10815600802090015AE0FFB4031CAB530555E5554A
:10816600AA547002055414F9E59912851390015A20
:108176007404F0C29822EFB4042990018CE0FF0445
:10818600F074632FF582E43401F583E599F0C29823
:1081960090018CE0B4281C90018E7401F0E49001EB
:1081A6005AF022C2982230990AC299900159E07079
:0481B60002C255228A
:1098F3002051221279BF43E740754A0AE4F54990A3
:109903000159F090015AF0C250D2517584017598F3
:0699130090C29CF59922B0
:108EFE0090018DE0705C9001ABE0FF7025D3900186
:108F0E0060E0948690015FE094674008E4F0A374FB
:108F1E0002F0800E900160E02428F090015FE034B2
:108F2E0000F0900160E02FFF90015FE03400FE1230
:108F3E0073B79001ABE02463F582E43401F583EF5F
:108F4E00F09001ABE004F0E0B42807E4F090018D5E
:038F5E0004F022FA
:108A7A0090018EE0607A900161E0FEA3E0FFC3946A
:108A8A0002EE94005006E490018EF0229001ABE0D1
:108A9A007C002FFFEC3EFE1273B79001ABE024631B
:108AAA00F582E43401F583E0FD6F60179001ABE0D5
:108ABA00FF900162E02FFF900161E03400FE127323
:108ACA0076D2549001ABE004F0E0B42823E490019C
:108ADA008EF09001ABF0900161E07004A3E06402B3
:108AEA00700E30540BC254128739128FC112901D66
:018AFA002259
:108DC9003050647584019001A0E0B40D00505590B5
:108DD9008DDFF8282873028E06028E09028E0C0296
:108DE9008E0F028E12028E15028E18028E1B028EB3
:108DF9001E028E21028E24028E27028E2A0298409C
:108E0900029A550293E00295E302991902005E0263
:108E1900980D02973A02961F0294230299F4029838
:088E29009B0299D9129A0E2256
:109840007897E67028759898754A0AF54990005BF4
:10985000E0B401079001A07404F022E490015AF0F2
:0E986000900159F09001A0E004F01279B922B5
:109A550090015A7401F0E4900159F0C2559001A0AB
:049A6500E004F02207
:1093E00090005BE01475F005A4B54919E4B5F015DB
:1093F0007598981279BFE4900159F090015AF09055
:1094000001A07404F0E54975F00584AFF0BF0112C6
:10941000C256E4900159F090015A04F09001A0E086
:0394200004F02233
:1095E300E54975F00584AFF0BF043020561EE54908
:1095F30075F00584FF24EFF582E43400F583E4F08D
:1096030074042FF582E43401F583E4F0E490015906
:0C961300F090015AF09001A0E014F02249
:1099190090005BE075F005A424FDB549159000524F
:10992900E0F599E4900159F090015AF09001A0E016
:0399390004F02215
:0D005E00900053E0F5999001A0E004F0221D
:10980D0090005BE0FD75F005A4FFE549B50723E485
:10981D00B5F01FEDB414079001A07409F022127970
:10982D00B9E4900159F0C25590015AF09001A0E0B1
:03983D0004F02212
:10973A00E549B464121279BFE4900159F090015AD4
:10974A00F09001A07409F0E54975F00584AFF0BF07
:10975A000112C256E4900159F090015A04F09001A6
:05976A00A0E004F02264
:10961F00E54975F00584AFF0BF043020561EE549CB
:10962F0075F00584FF24EFF582E43400F583E4F050
:10963F0074042FF582E43401F583E4F0E4900159CA
:0C964F00F090015AF09001A0E014F0220D
:10942300E5496465703C90018DE0B4012F755301EB
:1094330075540175555FE4900159F090015AF07528
:109443008401AB530555E555AA547002055414F92C
:109453001284CDF5999001A0E004F0229001A0744C
:039463000CF022E8
:1099F400758401AB53AA54A9551284CDF599E4900A
:0A9A0400018BF09001A0E004F022B5
:10989B0075840190018BE0FF04F074632FF582E473
:1098AB003401F583E0F59990018BE0D39428400BBC
:0C98BB00E490018DF09001A0E004F02288
:1099D900E549B46915C250C251E49000EDF0900117
:0B99E90059F090015AF09001A0F0220C
:109A0E00C250C251E4F5499000EDF0900159F0902A
:089A1E00015AF09001A0F022B2
:1090D2003052527584019001A1E0B40A00504390CD
:1090E20090E8F828287302910602910902910C0275
:1090F200910F02911202911502911802911B029195
:109102001E02912102970402965B02969402999C98
:10911200029AC50298C70294EB0296CC02993C02CD
:069122009AB4129AD52256
:10970400E549703175989890005BE0B401131279C3
:10971400BFE490015AF0900159F09001A17403F054
:10972400221279B9C255E490015AF0900159F0908F
:0697340001A1E004F02297
:10965B0090005BE01475F005A4B54911E4B5F00D6D
:10966B007598981279BF9001A17403F022E54975A2
:10967B00F00584AFF0BF0110C256C25590015A7469
:09968B0001F09001A1E004F022BD
:10969400E54975F00584AFF0BF042C20561EE5495A
:1096A40075F00584FF24EFF582E43400F583E4F0DB
:1096B40074042FF582E43401F583E4F0E490015A54
:0896C400F09001A1E014F02276
:10999C0090005BE075F005A424FDB54911758401B8
:0F99AC00900052E0F599C2559001A1E004F0221D
:109AC500758401900053E0F5999001A1E004F0221E
:1098C70090005BE0FFB414079001A17406F022EF4B
:1098D70075F005A4B54914E4B5F0101279B99001F3
:0C98E700A1E004F0C255E490015AF02208
:1094EB00E54975F00584AFF0BF0111C256C2559026
:1094FB00015A7401F09001A1E004F022E549B46433
:10950B001F1279B990018EE0700B90015AF0900107
:10951B00A17408F022E490015AF09001A17409F0B3
:01952B00221D
:1096CC00E54975F00584AFF0BF042C20561EE54922
:1096DC0075F00584FF24EFF582E43400F583E4F0A3
:1096EC0074042FF582E43401F583E4F0E490015A1C
:0896FC00F09001A1E014F0223E
:10993C00E549B4651A755301755401755561E49088
:10994C00018CF09001A17409F090015A7402F0227C
:109AB400E549B4690BC252E490015AF09001A1F057
:019AC400227F
:109AD500C252E490015AF0900159F09001A1F02290
:1081BA00789AE6600116900000E0600214F09000E0
:1081CA0001E0600214F0900002E0600214F09000F6
:1081DA000BE0600214F090000AE0600214F0789C50
:1081EA0016E6600302828D789C760A789BE6600127
:1081FA0016900004E0600214F0900005E06002149A
:10820A00F0900006E0600214F0900008E0600214AA
:10821A00F0900009E0600214F078A0E66001169080
:10822A000003E0600214F09001E7E0600214F078C5
:10823A009D16E6704E789D760A90000CE060021456
:10824A00F078A2E61846600708E61618700116903C
:10825A0001A3E0600214F09001A4E0600214F0901F
:10826A0001A7E0600214F0789E16E67016789E76F2
:10827A000A789F16E6700C789F76069001A6E06051
:04828A000214F022C8
:106B2200535155452020434F53202053454E534542
:106B3200004F4E2020202020202020202020202016
:106B420020004F46462020202020202020202020E8
:106B520020200020202052455045415445522031EA
:106B620020202000202020524550454154455220EB
:106B720032202020002020205245504541544552C9
:106B820020332020200020202052455045415445EA
:106B920052203420202000202020524550454154CC
:106BA20045522035202020002020205245504541CA
:106BB20054455220362020200020202052455045A6
:106BC2004154455220372020200020202052455099
:106BD2004541544552203820202000202020524593
:106BE2005045415445522039202020002020205277
:106BF200455045415445522031302020002020206C
:106C02005245504541544552203131202000202028
:106C12002052455045415445522031322020002017
:106C22002020524550454154455220313320200006
:106C320020202052455045415445522031342020D5
:106C420000202020524550454154455220313520E4
:106C520020002020205245504541544552203136D3
:106C620020200020202052455045415445522031D9
:106C720037202000202020524550454154455220C3
:106C820031382020002020205245504541544552A1
:106C920020313920200020202052455045415445C2
:076CA20052203230202000D7
:10002E00750C01E50CC394155018AF0C74182FF510
:10003E0082E43401F583E0FFEF60037F0122050CBB
:04004E0080E17F00CE
:01005200228B
:1090790020575512835CEF6401704D90009AE0FF10
:10908900EF24FF924D900158E0FF74422FF582E4DE
:109099003401F583E0FF90015BEFF0900158E0FFA8
:1090A900742D2FF582E43401F583E0FF90015CEF24
:1090B900F0900158E0FF90015DEFF01264629001B9
:0990C9005EEFF0128573D23F2224
:10835C009000E8E4F0A3E4F09000EBE4F0A3E4F088
:10836C009000E7E4F09000E7E0FFEFC394154003C2
:10837C00028400900158E0FFEFD394144006900162
:10838C00587401F0900158E0FF74182FF582E43412
:10839C0001F583E0FF9000EAEFF09000EAE0FFEFD8
:1083AC00B40115900158E0FF74182FF582E43401E4
:1083BC00F5837402F07F01229000EAE0FFEFB40233
:1083CC00249000E8E0FEA3E0FFEF4E70189000E868
:1083DC00E4F0A37401F0900158E0FF7E009000EBF4
:1083EC00EEF0A3EFF0900158E004F09000E7E00409
:1083FC00F00283719000E8E0FEA3E0FFEF4E700402
:10840C007F0022229000ECE0FF900158EFF07F01FA
:01841C00223D
:10828E009000E8E4F0A3E4F09000EBE4F0A3E4F057
:10829E009000E7E4F09000E7E0FFEFC39415400391
:1082AE0002833F900158E0FFEFD3941440069001F3
:1082BE00587401F0900158E0FF74182FF582E434E1
:1082CE0001F583E0FF9000EAEFF09000EAE0FFEFA7
:1082DE00605090005BE0FF900158E0FEEE6F604250
:1082EE009000EAE0FFEFB40115900158E0FF74181A
:1082FE002FF582E43401F5837402F07F01229000A1
:10830E00E8E0FEA3E0FFEF4E7018900158E0FF7E0C
:10831E00009000EBEEF0A3EFF09000E8E4F0A37411
:10832E0001F0900158E004F09000E7E004F00282C2
:10833E00A39000E8E0FEA3E0FFEF4E70047F002262
:0E834E00229000ECE0FF900158EFF07F01223A
:1064620090005BE0FFEFD3941440037F2022900161
:10647200EDE4F09001ECE4F090005BE0FF9001EAC3
:10648200EFF0900095E0FFEFD394065003026556BB
:106492009001EBE4F09001EBE0FFEFC394154003B1
:1064A20002654F9001EAE0FFEFB415069001EA742D
:1064B20001F09001EAE0FF74EE2FF582E43400F57A
:1064C20083E0FFEF64FF70769001EAE0FF74BE2F75
:1064D200F582E43400F583E0FF90005BE0FE74BED9
:1064E2002EF582E43400F583E0FEEEC39F404F9028
:1064F200005BE0FF9001EAE0FEEEB507069001EADC
:10650200E0FF229001EAE0FF74BE2FF582E434003E
:10651200F583E0FF9001ECE0FEEFD39E4020900176
:10652200EAE0FF9001EDEFF09001EAE0FF74BE2F88
:10653200F582E43400F583E0FF9001ECEFF0900186
:10654200EBE004F09001EAE004F00264979001EDC0
:10655200E0FF22229001EBE4F09001EBE0FFEFC3B9
:10656200941540030266129001EAE0FFEF70069074
:1065720001EA7414F09001EAE0FF74EE2FF582E470
:106582003400F583E0FFEF64FF70769001EAE0FFEC
:1065920074BE2FF582E43400F583E0FF90005BE0E7
:1065A200FE74BE2EF582E43400F583E0FEEEC39F56
:1065B200404F90005BE0FF9001EAE0FEEEB5070677
:1065C2009001EAE0FF229001EAE0FF74BE2FF5821B
:1065D200E43400F583E0FF9001ECE0FEEFD39E404F
:1065E200209001EAE0FF9001EDEFF09001EAE0FF78
:1065F20074BE2FF582E43400F583E0FF9001ECEFE6
:10660200F09001EBE004F09001EAE014F002655B27
:056612009001EDE0FF26
:016617002260
:1069820090005BE0FFEFD3941440037F202290013C
:10699200F1E4F09001F0E4F0900095E0FFEFD39481
:1069A200065003026A6790005BE0FFEF04FF90016C
:1069B200EEEFF09001EFE4F09001EFE0FFEFC3940F
:1069C200154003026A609001EEE0FFEFD394144099
:1069D200069001EE7401F09001EEE0FF74EE2FF5E7
:1069E20082E43400F583E0FFEF64FF70629001EE11
:1069F200E0FF74BE2FF582E43400F583E0FF9000DF
:106A02005BE0FE74BE2EF582E43400F583E0FEEE18
:106A1200C39F403B9001EEE0FF74BE2FF582E43449
:106A220000F583E0FF9001F0E0FEEFD39E4020905E
:106A320001EEE0FF9001F1EFF09001EEE0FF74BE95
:106A42002FF582E43400F583E0FF9001F0EFF0903F
:106A520001EFE004F09001EEE004F00269BA900167
:106A6200F1E0FF222290005BE0FFEF14FF9001EEC5
:106A7200EFF09001EFE4F09001EFE0FFEFC3941527
:106A82004003026B1C9001EEE0FFEF70069001EEF6
:106A92007414F09001EEE0FF74EE2FF582E43400FE
:106AA200F583E0FFEF64FF70629001EEE0FF74BED9
:106AB2002FF582E43400F583E0FF90005BE0FE7482
:106AC200BE2EF582E43400F583E0FEEEC39F403B28
:106AD2009001EEE0FF74BE2FF582E43400F583E00E
:106AE200FF9001F0E0FEEFD39E40209001EEE0FF28
:106AF2009001F1EFF09001EEE0FF74BE2FF582E419
:106B02003400F583E0FF9001F0EFF09001EFE00434
:0F6B1200F09001EEE014F0026A799001F1E0FFDB
:016B21002251
:1067CD0090005BE0FFEFD3941440037F20229000F4
:1067DD0052E0FFEFB4FF0C900053E0FFEFB4FF0366
:1067ED007F00229001F5E4F09001F4E4F090009523
:1067FD00E0FFEFD3940650030268C790005BE0FF03
:10680D00EF04FF9001F2EFF09001F3E4F09001F34B
:10681D00E0FFEFC3941540030268C09001F2E0FF62
:10682D00EFD3941440069001F27401F09001F2E060
:10683D00FF74EE2FF582E43400F583E0FFEF64FF83
:10684D0070629001F2E0FF74BE2FF582E43400F522
:10685D0083E0FF90005BE0FE74BE2EF582E4340011
:10686D00F583E0FEEEC39F403B9001F2E0FF74BE66
:10687D002FF582E43400F583E0FF9001F4E0FEEFA4
:10688D00D39E40209001F2E0FF9001F5EFF09001D2
:10689D00F2E0FF74BE2FF582E43400F583E0FF9043
:1068AD0001F4EFF09001F3E004F09001F2E004F058
:1068BD0002681A9001F5E0FF222290005BE0FFEFE5
:1068CD0014FF9001F2EFF09001F3E4F09001F3E08A
:1068DD00FFEFC39415400302697C9001F2E0FFEFD6
:1068ED0070069001F27414F09001F2E0FF74EE2F37
:1068FD00F582E43400F583E0FFEF64FF70629001F0
:10690D00F2E0FF74BE2FF582E43400F583E0FF90D2
:10691D00005BE0FE74BE2EF582E43400F583E0FEEC
:10692D00EEC39F403B9001F2E0FF74BE2FF582E471
:10693D003400F583E0FF9001F4E0FEEFD39E40209C
:10694D009001F2E0FF9001F5EFF09001F2E0FF749D
:10695D00BE2FF582E43400F583E0FF9001F4EFF0F3
:10696D009001F3E004F09001F2E014F00268D99088
:04697D0001F5E0FF41
:0169810022F3
:109A690090005BE0FFEFD3941440037F2022900025
:049A79005BE0FF228D
:10785B00900157E0FFEFD394144006900157740149
:10786B00F09000E7E4F0900157E0FF742D2FF582C4
:10787B00E43401F583E0FF900157E0FE74032EF52D
:10788B0082E43401F583E0FEEEB50726900157E064
:10789B00FF74422FF582E43401F583E0FF9001572A
:1078AB00E0FE74EE2EF582E43400F583E0FEEE6F1D
:1078BB0060069000E77401F0900157E0FF74EE2F23
:1078CB00F582E43400F583E0FF90005BE0FEEF6EA1
:1078DB00600E90005BE0FF900157E0FEEE6F703A98
:1078EB009000E7E0FFEF6043900157E0FFEFD39488
:1078FB00155014900157E0FF74182FF582E43401F2
:10790B00F5837401F08024900157E0FF74182FF574
:10791B0082E43401F583E4F08011900157E0FF74A9
:10792B00182FF582E43401F583E4F09000E7E0FFD3
:10793B00EF6044900157E0FF74032FF582E43401AC
:10794B00F583E0FF900157E0FE742D2EF582E434B1
:10795B0001F583EFF0900157E0FF74EE2FF582E411
:10796B003400F583E0FF900157E0FE74422EF58260
:0E797B00E43401F583EFF0900157E004F022B0
:10722200900198E0FFEF60030272D0900006E0FF49
:10723200EF70037F01221294A9EFB4010512799B2A
:1072420080031279A1204A037F00221294A9EF64DD
:10725200017078304A72C24A1270CB90004EE0FF41
:10726200900194EFF090004FE0FF900195EFF090C5
:10727200004DE0FF900196EFF0900196E0FFEFB431
:107282001F14900192E0FF900195E0FEEEB5070613
:107292001279A17F0122900191E0FF900194E0FE1A
:1072A200EEB5070E900192E0FF900195E0FEEE6FC1
:1072B20060099001987401F07F002290008CE0FF39
:1072C200900006EFF07F00227F00227F00229001D3
:1072D20098E0FFEF6401600302736E900006E0FF26
:1072E200EF70037F01221294A9EFB4010512799B7A
:1072F20080031279A1204A037F0022C24A1270CB76
:1073020090004EE0FF900194EFF090004FE0FF906C
:107312000195EFF090004DE0FF900196EFF09001A3
:1073220096E0FFEFB41F14900192E0FF900195E008
:10733200FEEEB507061279A17F0122900191E0FFCE
:10734200900194E0FEEEB50720900192E0FF9001DB
:1073520095E0FEEEB5071290008CE0FF900006EF7C
:10736200F0900198E4F07F00227F0022900198E4DF
:04737200F07F002286
:1094A900900083E0FFEF600D1279C540047F0180D1
:1094B900027F002222900084E0FFEF601390008574
:1094C900E0FFE532D39F40047F0122227F00222260
:1094D900900085E0FFE532C39F50047F0122227F7F
:0294E90000225F
:106F6F0090019DE0FFEF6003027021900008E0FFA9
:106F7F00EF70037F01221294A9EFB4010512799BE0
:106F8F0080031279A190019CE0FFEFB40106203B32
:106F9F00037F002290019CE0FFEFB4020620410323
:106FAF007F00221294A9EF6401706490019CE0FFAE
:106FBF00EF64017021303B1EC23BE53F653E600927
:106FCF0090019D7401F07F0022900091E0FF9000EE
:106FDF0008EFF07F002290019CE0FFEF6402702F1A
:106FEF0030412CC24190019FE534F090019FE0FFAA
:106FFF0090019EE0FEEE6F600990019D7401F07F9D
:10700F000022900091E0FF900008EFF07F00227FB8
:10701F00002290019DE0FFEF640160030270CA90AF
:10702F000008E0FFEF70037F01221294A9EFB40173
:10703F000512799B80031279A190019CE0FFEFB4B8
:10704F000106203B037F002290019CE0FFEFB4027A
:10705F00062041037F00221294A9EF6401705A9019
:10706F00019CE0FFEFB4011C303B19C23BE53FB57B
:10707F003E1290019DE4F0900091E0FF900008EF28
:10708F00F07F002290019CE0FFEF6402702B3041F3
:10709F0028C24190019FE534F090019FE0FF9001DD
:1070AF009EE0FEEEB5071290019DE4F0900091E096
:0C70BF00FF900008EFF07F00227F00220D
:108E31007BFF7A6B792212976F1279C5400B7BFF0A
:108E41007A6B79331297A480097BFF7A6B7944128C
:108E510097A47F17127DB6AF32127A6C900054E05E
:108E6100FF127D87900055E0FF127D87900056E04C
:108E7100FF127D877F1C127DB6AF31127A6C900094
:108E810054E0FF127D87900055E0FF127D8790002E
:078E910056E0FF127D87226D
:10986E00900088E0FFEF6013900089E0FFE531D3B0
:10987E009F40047F0122227F002222900089E0FF78
:0D988E00E531C39F50047F0122227F00229C
:109AE500900083E0FFEF6004128AFB22126CA9222A
:108AFB009001A5E0FFEF70161279C54072900086C9
:108B0B00E0FF90000AEFF09001A5E004F022900145
:108B1B00A5E0FFEF640170281279C5401C90000A94
:108B2B00E0FFEF704AD25B900090E0FF900007EF00
:108B3B00F09001A5E004F022229001A5E4F022229E
:108B4B009001A5E0FFEFB402211279C5400B900014
:108B5B0090E0FF900007EFF022900007E0FFEF702E
:108B6B000EC25B9001A5E4F022229001A5E4F02255
:106CA9009001A5E0FFEF704C900084E0FFEF6023B6
:106CB900900085E0FFE532D39F4013900086E0FF06
:106CC90090000AEFF09001A5E004F0228026C25B53
:106CD900228021900085E0FFE532C39F5013900088
:106CE90086E0FF90000AEFF09001A57403F022807E
:106CF90003C25B229001A5E0FFEF640170359000AB
:106D090085E0FFEF24FBFFE532D39F401F90000A87
:106D1900E0FFEF6003026E0CD25B900087E0FF900A
:106D2900000BEFF09001A5E004F022229001A5E408
:106D3900F022229001A5E0FFEF6402702E900085F9
:106D4900E0FFEF24FBFFE532D39F400B900087E083
:106D5900FF90000BEFF02290000BE0FFEF600302C1
:106D69006E0CC25B9001A5E4F022229001A5E0FF20
:106D7900EF64037043900085E0FF7E00EF2405FF78
:106D8900EE3400FEAD327C00C3ED9FEE6480F8EC7A
:106D9900648098501C90000AE0FFEF7066D25B9007
:106DA9000087E0FF90000BEFF09001A5E004F022CE
:106DB900229001A5E4F022229001A5E0FFEF6404EE
:106DC900703C900085E0FF7E00EF2405FFEE340063
:106DD900FEAD327C00C3ED9FEE6480F8EC648098D0
:106DE900500B900087E0FF90000BEFF02290000B12
:106DF900E0FFEF700EC25B9001A5E4F02222900142
:046E0900A5E4F022EA
:109A26001267CD8F1D9001E6E0FFEF651D6008907F
:079A360001E6E51DF0D25C22
:019A3D002206
:107BD30090005BE0FFEF12854D7C1C017C26027C4C
:107BE30030037C3A047C44057C4E067C58077C6257
:107BF300087C6C097C760A7C800B7C8A0C7C940D57
:107C03007C9E0E7CA80F7CB2107CBC117CC6127CBF
:107C1300D0137CDA1400007CE37BFF7A6B79551276
:107C230097A4227BFF7A6B79661297A4227BFF7A53
:107C33006B79771297A4227BFF7A6B79881297A4CA
:107C4300227BFF7A6B79991297A4227BFF7A6B7957
:107C5300AA1297A4227BFF7A6B79BB1297A4227B8B
:107C6300FF7A6B79CC1297A4227BFF7A6B79DD12B2
:107C730097A4227BFF7A6B79EE1297A4227BFF7A7B
:107C83006B79FF1297A4227BFF7A6C79101297A469
:107C9300227BFF7A6C79211297A4227BFF7A6C797D
:107CA300321297A4227BFF7A6C79431297A4227B2A
:107CB300FF7A6C79541297A4227BFF7A6C79651250
:107CC30097A4227BFF7A6C79761297A4227BFF7AA2
:107CD3006C79871297A4227BFF7A6C79981297A408
:017CE300227E
:105660002020464C455820495620303036202020F6
:10567000002049502050524F4752414D4D494E470E
:10568000200043544353532036332E302020202013
:10569000202043544353532036372E3020202020DF
:1056A000202043544353532036392E3420202020C9
:1056B000202043544353532037312E3920202020BB
:1056C000202043544353532037342E3420202020AD
:1056D000202043544353532037372E30202020209E
:1056E000202043544353532037392E372020202085
:1056F000202043544353532038322E35202020207D
:10570000202043544353532038352E34202020206A
:10571000202043544353532038382E352020202056
:10572000202043544353532039312E35202020204C
:10573000202043544353532039342E382020202036
:10574000202043544353532039372E342020202027
:1057500020204354435353203130302E302020201A
:1057600020204354435353203130332E3520202002
:1057700020204354435353203130372E32202020F1
:1057800020204354435353203131302E39202020E0
:1057900020204354435353203131342E38202020CD
:1057A00020204354435353203131382E38202020B9
:1057B00020204354435353203132332E30202020B5
:1057C00020204354435353203132372E332020209E
:1057D00020204354435353203133312E382020208E
:1057E00020204354435353203133362E352020207C
:1057F00020204354435353203134312E3320202072
:1058000020204354435353203134362E322020205D
:1058100020204354435353203135312E342020204F
:1058200020204354435353203135362E3720202037
:1058300020204354435353203135392E3820202023
:1058400020204354435353203136322E322020201F
:1058500020204354435353203136352E3520202009
:1058600020204354435353203136372E39202020F3
:1058700020204354435353203137312E33202020EE
:1058800020204354435353203137332E38202020D7
:1058900020204354435353203137372E33202020C8
:1058A00020204354435353203137392E39202020B0
:1058B00020204354435353203138332E35202020A9
:1058C00020204354435353203138362E3220202099
:1058D00020204354435353203138392E392020207F
:1058E00020204354435353203139322E3820202076
:1058F00020204354435353203139362E3620202064
:1059000020204354435353203139392E3520202051
:1059100020204354435353203230332E352020204F
:1059200020204354435353203230362E352020203C
:1059300020204354435353203231302E372020202F
:1059400020204354435353203231382E312020201D
:1059500020204354435353203232352E3720202009
:1059600020204354435353203232392E31202020FB
:1059700020204354435353203233332E36202020EB
:1059800020204354435353203234312E38202020DA
:1059900020204354435353203235302E33202020CF
:1059A00020204354435353203235342E31202020BD
:1059B00020202020202020202020202020202020E7
:0259C0002020A5
:1062A60075840F1266189001E87401F09001E97484
:1062B60003F07D007CFC7F10129569E49001E8F004
:1062C6009001E9F020A10875840F43E8C0800675A7
:1062D600840F53E83F129AF57BFF7A56796012973E
:1062E6006F129A3E900003741EF0900003E070FA5D
:1062F600129AA290005BE0FF6005D39414400690CA
:10630600005B7401F0127BD3128739128FC1129091
:106316001D1297D9D2AC12798F900099E0FF78A11F
:10632600760008A6079000A4E09001A6F0E490008D
:10633600EDF0900190F090018FF0900198F09001AF
:10634600A0F090005274FFF0900053F0E49001E644
:10635600F09001E5F0F5581279A1304313124AEF97
:10636600129AA2128739128FC112901DC24380EA77
:1063760020A60E128E31E4900190F090018FF080ED
:10638600EF30461DC246124AEF129AA21287391200
:106396008FC112901D129AF5E490018FF090019032
:1063A600F043E740305806128EFE1298F312425020
:1063B6001232E81275EFE55BB45514E55CB4AA0F2A
:1063C6009001E77414F09001E7E070FA1279959065
:1063D60001A7E0703E1279A75039127AB512785BA0
:1063E600125AA6129AE5128F61129A26305C8130F3
:1063F6005D03026376C25C9001E6E02400FEE434AD
:10640600179001C2F0A3CEF09001BE7401F0D25DE8
:1064160002637612798F900099E0FF78A1760008E2
:10642600A6079000A4E09001A6F0E49000EDF0909D
:106436000190F090018FF0900198F09001A0F090FB
:10644600005BE0900052F090005374FCF01279A1CA
:0C6456007BFF7A56797112976F02637613
:108E980001AE01C901DA01EB01FC020E0220023326
:108EA8000247025C02710287029902AB02C302DC2C
:108EB80002F50310032B03480365038403A403C5C9
:108EC80003E6040A042E04430453046A047A049152
:108ED80004A204BA04CC04E504F705100524053EF1
:108EE8000552056D0582059E05D10605061C063B43
:068EF800067306AD06C77B
:1099BB00C23DC23FEF25E02498F582E4348EF58357
:0E99CB00E493F51A740193F51BD23ED23822B4
:09009600C23DC23FC23EC2382245
:0300A3000294665E
:10946600C0E0C0F0C083C082C0D075D000C000C0CC
:1094760001C002C003C004C005C006C007205805CD
:109486001280E68003129128D007D006D005D004BA
:10949600D003D002D001D000D0D0D082D083D0F07B
:0394A600D0E032E1
:03009300028CF4E8
:0B8CF400C0E0C0D075D000C006C00773
:108CFF00AE84758402E5337007AFBE75BB07802F56
:108D0F00E533B40107AFBE75BB048023E533B4026E
:108D1F0007AFBE75BB068017E533B4030885BE31B8
:108D2F0075BB04800AE533B40409AFBE75BB0505F6
:108D3F00338010E533B4050885BE3275BB0480005F
:078D4F00753300C2ED8E84B4
:098D5600D007D006D0D0D0E032E5
:0300830002952CB7
:10952C00C0E0C0F0C083C082C0D075D000C000C005
:10953C0001C002C003C004C005C006C007C2CF12E0
:10954C001D32D007D006D005D004D003D002D001F4
:0D955C00D000D0D0D082D083D0F0D0E0324B
:0300730002885DA3
:10885D00C0E0C0F0C083C082C0D075D000C000C0E1
:10886D0001C002C003C004C005C006C007C2CF309E
:10887D005805128DC980031290D27897E6600116C3
:10888D00304027C240D54A05754A0A05491274B3CE
:10889D00D51C09751C0A758401438820D5301875BF
:1088AD003060758402438820800DD240789816E69A
:1088BD0070057604121A1A758401438810758402A6
:1088CD00D2ECD007D006D005D004D003D002D00111
:0D88DD00D000D0D0D082D083D0F0D0E032D7
:03006B0002930FEE
:10930F00C0E0C0F0C083C082C0D075D000C000C024
:0D931F0001C002C003C004C005C006C007A5
:0E932C008584741281BA758402C28D857484A2
:10933A00D007D006D005D004D003D002D001D00087
:0B934A00D0D0D082D083D0F0D0E03231
:03005B00029224EA
:10922400C0E0C0F0C083C082C0D075D000C000C010
:1092340001C002C003C004C005C006C0071259DB48
:109244007899E6600116900007E0600214F07584D6
:1092540001C28D1277D1D007D006D005D004D00337
:10926400D002D001D000D0D0D082D083D0F0D0E0D2
:0192740032C7
:03005300029355C0
:10935500C0E0C0F0C083C082C0D075D000C000C0DE
:1093650001C002C003C004C005C006C007C28C30DE
:109375005904C2598005D2591274D5D007D006D0E8
:1093850005D004D003D002D001D000D0D0D082D0F7
:0693950083D0F0D0E032AD
:03002B00020016BA
:03001600C2CF3224
:03002300029A90AE
:109A9000309904C299C262309807859956C298D20B
:029AA000613231
:03001B00020019C7
:0100190032B4
:10939B00A984A2AF9264AEB1C2AF75840F53A1FE84
:1093AB008FB1E4F5849001E8E042B79001E9E04227
:1093BB008F8C088D098D828C83EBF0E4F584900102
:1093CB00E9E0F4528F9001E8E0F452B78EB1898452
:0493DB00A26492AF47
:0193DF00226B
:10956900A984A2AF9264AEB1C2AF8C088D098FB144
:10957900E4F5849001E8E0FF42B7E4F5849001E95D
:10958900E0FD428F850982850883E4F0EDF4528F6E
:0C959900EFF452B78EB18984A26492AF47
:0195A50022A3
:10995C00AE84A2AF9264ABB1C2AF8FB18C0A8D0B47
:0F996C008D828C83E493FF8BB18E84A26492AFC3
:01997B0022C9
:100EC800202020464C45582049562020202020200C
:100ED8000020202020202020202020202049444CB1
:100EE80045002054657374696E67204D6F646520F2
:100EF80020200043726F73732042757379204D6F01
:100F08006465200053656E642049646C654D6573A3
:100F1800736167650043726F73732042757379203C
:100F28004D6F6465310043726F7373204275737936
:100F3800204D6F6465320043726F7373204275737E
:100F480079204D6F6465330043726F737320427567
:100F58007379204D6F64653400202053656E646991
:100F68006E672043574944202000205741495420A8
:100F78005544544420464C414720004C5452564F47
:100F88004950204F5554474F494E470020564F4926
:100F980050204F5554474F494E47202000202049A4
:100FA8004E434F4D494E47204C545220200020209C
:100FB800494E434F4D494E472043544353532020F5
:100FC800002020494E434F4D494E4720444353206B
:100FD800200043544353532036332E302020202002
:100FE800202043544353532036372E3020202020CE
:100FF800202043544353532036392E3420202020B8
:10100800202043544353532037312E3920202020A9
:10101800202043544353532037342E34202020209B
:10102800202043544353532037372E30202020208C
:10103800202043544353532037392E372020202073
:10104800202043544353532038322E35202020206B
:10105800202043544353532038352E342020202059
:10106800202043544353532038382E352020202045
:10107800202043544353532039312E35202020203B
:10108800202043544353532039342E382020202025
:10109800202043544353532039372E342020202016
:1010A80020204354435353203130302E3020202009
:1010B80020204354435353203130332E35202020F1
:1010C80020204354435353203130372E32202020E0
:1010D80020204354435353203131302E39202020CF
:1010E80020204354435353203131342E38202020BC
:1010F80020204354435353203131382E38202020A8
:1011080020204354435353203132332E30202020A3
:1011180020204354435353203132372E332020208C
:1011280020204354435353203133312E382020207C
:1011380020204354435353203133362E352020206A
:1011480020204354435353203134312E3320202060
:1011580020204354435353203134362E322020204C
:1011680020204354435353203135312E342020203E
:1011780020204354435353203135362E3720202026
:1011880020204354435353203135392E3820202012
:1011980020204354435353203136322E322020200E
:1011A80020204354435353203136352E35202020F8
:1011B80020204354435353203136372E39202020E2
:1011C80020204354435353203137312E33202020DD
:1011D80020204354435353203137332E38202020C6
:1011E80020204354435353203137372E33202020B7
:1011F80020204354435353203137392E392020209F
:1012080020204354435353203138332E3520202097
:1012180020204354435353203138362E3220202087
:1012280020204354435353203138392E392020206D
:1012380020204354435353203139322E3820202064
:1012480020204354435353203139362E3620202052
:1012580020204354435353203139392E3520202040
:1012680020204354435353203230332E352020203E
:1012780020204354435353203230362E352020202B
:1012880020204354435353203231302E372020201E
:1012980020204354435353203231382E312020200C
:1012A80020204354435353203232352E37202020F8
:1012B80020204354435353203232392E31202020EA
:1012C80020204354435353203233332E36202020DA
:1012D80020204354435353203234312E38202020C9
:1012E80020204354435353203235302E33202020BE
:1012F80020204354435353203235342E31202020AC
:1013080020202020202020202020202020202020D5
:1013180020204443532030303620494E5620303266
:1013280031204443532030303720494E5620323143
:1013380034204443532030313520494E562031342F
:1013480031204443532030313720494E5620303520
:1013580030204443532030323120494E562030301B
:1013680036204443532030323320494E56203034FF
:1013780037204443532030323520494E56203234EA
:1013880034204443532030323620494E56203436D8
:1013980034204443532030333120494E56203632CE
:1013A80037204443532030333220494E56203035BD
:1013B80031204443532030333620494E56203137AC
:1013C80032204443532030343320494E562034349D
:1013D80035204443532030343720494E562030328C
:1013E80033204443532030353020494E5620303185
:1013F80037204443532030353120494E562030336E
:1014080032204443532030353320494E562034355A
:1014180032204443532030353420494E562034314D
:1014280033204443532030363520494E5620323736
:1014380031204443532030373120494E5620333031
:1014480036204443532030373220494E5620323418
:1014580035204443532030373320494E5620353009
:1014680036204443532030373420494E56203137F4
:1014780034204443532031313420494E56203731EB
:1014880032204443532031313520494E56203135DE
:1014980032204443532031313620494E56203735C7
:1014A80034204443532031323220494E56203232C0
:1014B80035204443532031323520494E56203336A7
:1014C80035204443532031333120494E562033369A
:1014D80034204443532031333220494E562035348A
:1014E80036204443532031333420494E562032327B
:1014F80033204443532031343120494E5620303173
:1015080035204443532031343320494E562034315A
:1015180032204443532031343520494E5620323747
:1015280034204443532031353220494E562031313E
:1015380035204443532031353520494E5620373322
:1015480031204443532031353620494E5620323617
:1015580035204443532031363220494E5620353009
:1015680033204443532031363520494E56203235F6
:1015780031204443532031373220494E56203033EE
:1015880036204443532031373420494E56203037D3
:1015980034204443532032303520494E56203236C9
:1015A80033204443532032313220494E56203335BC
:1015B80036204443532032313420494E56203030AF
:1015C80037204443532032323320494E562031339A
:1015D80034204443532032323520494E562031328C
:1015E80032204443532032323620494E562034317B
:1015F80031204443532032343320494E562033356A
:1016080031204443532032343420494E562030325E
:1016180035204443532032343520494E5620303744
:1016280032204443532032343620494E5620353236
:1016380033204443532032353120494E5620313629
:1016480035204443532032353220494E5620343613
:1016580032204443532032353520494E5620343405
:1016680036204443532032363120494E56203733F2
:1016780032204443532032363320494E56203230EC
:1016880035204443532032363520494E56203135D3
:1016980036204443532032363620494E56203435BE
:1016A80034204443532032373120494E56203036B7
:1016B80035204443532032373420494E56203134A4
:1016C80035204443532033303620494E5620303796
:1016D80031204443532033313120494E5620363689
:1016E80034204443532033313520494E5620343278
:1016F80033204443532033323520494E5620353267
:1017080036204443532033333120494E5620343653
:1017180035204443532033333220494E5620343544
:1017280035204443532033343320494E5620353333
:1017380032204443532033343620494E5620363124
:1017480032204443532033353120494E5620323419
:1017580033204443532033353620494E5620323106
:1017680032204443532033363420494E56203133F7
:1017780031204443532033363520494E56203132E8
:1017880035204443532033373120494E56203733D0
:1017980034204443532034313120494E56203232CC
:1017A80036204443532034313220494E56203134B8
:1017B80033204443532034313320494E56203035AA
:1017C80034204443532034323320494E5620333199
:1017D80035204443532034333120494E5620373284
:1017E80033204443532034333220494E5620353178
:1017F80036204443532034343520494E5620303463
:1018080033204443532034343620494E5620323551
:1018180035204443532034353220494E5620303544
:1018280033204443532034353420494E5620323631
:1018380036204443532034353520494E562033331F
:1018480032204443532034363220494E5620323514
:1018580032204443532034363420494E5620303207
:1018680036204443532034363520494E56203333EE
:1018780031204443532034363620494E56203636DC
:1018880032204443532035303320494E56203136D8
:1018980032204443532035303620494E56203037C5
:1018A80033204443532035313620494E56203433B3
:1018B80032204443532035323320494E56203234A7
:1018C80036204443532035323620494E5620333291
:1018D80035204443532035333220494E5620333483
:1018E80033204443532035343620494E5620313373
:1018F80032204443532035363520494E5620373060
:1019080033204443532036303620494E5620363350
:1019180031204443532036313220494E5620333447
:1019280036204443532036323420494E562036332D
:1019380032204443532036323720494E5620303324
:1019480031204443532036333120494E5620363017
:1019580036204443532036333220494E56203632FF
:1019680034204443532036353420494E56203734EA
:1019780033204443532036363220494E56203436DD
:1019880036204443532036363420494E56203331CE
:1019980031204443532037303320494E56203536C2
:1019A80035204443532037313220494E56203131B7
:1019B80034204443532037323320494E56203433A1
:1019C80031204443532037333120494E5620313596
:1019D80035204443532037333220494E562032367F
:1019E80031204443532037333420494E562033376F
:1019F80031204443532037343320494E562036355E
:101A080034204443532037353420494E5620313151
:021A1800362076
:107AB5009000B3E0FFB4010A90005274FFF0E402B5
:107AC5007B82EF64026003027B87127989787DE609
:107AD5006003027B76305703027B76900197E07056
:107AE50032D23F90009AE024FF924D90005BE0FF78
:107AF50090015BF0900098E090015CF090015DEFE3
:107B0500F012698290015EEFF0128573900197740F
:107B150002F02212828EEF64017050D23F9001581C
:107B2500E0FF2442F582E43401F583E090015BF047
:107B3500742D2FF582E43401F583E090015CF0901B
:107B45000158E090015DF012646290015EEFF090E3
:107B5500015BE024D2F582E43400F583E024FF9252
:107B65004D128573900197E014F022900197E0146F
:107B7500F090005BE0900052F0900098E090005388
:107B8500F02290018FE0B40900503D907B97F828D2
:107B95002873027BB2027BB5027BB8027BBB027BFA
:107BA500BE027BC1027BC4027BC7027BCA022537AA
:107BB5000289710287CC0252F30246B5022D680292
:0E7BC5003D5D024F00023850E490018FF02227
:10253700900190E0B40C004003022D6290254AF808
:1025470028287302256E0225A2022839022877025D
:10255700289A0228C402298A022A14022AA6022AD1
:10256700D3022B98022C6DE49001E5F07BFF7A0EE5
:1025770079C812976F7BFF7A0E79D91297A49000CA
:102587005274FFF0900053F012798F9000B4E0601E
:10259700031279B39001907401F02220A55C12799F
:1025A700899000B4E060031279AD9000B1E090002B
:1025B70000F090005BE0FF900052F0900098E0FE82
:1025C700900053F09001907405F090015BEFF0904C
:1025D700015CEEF090005BE090015DF012646290A8
:1025E700015EEFF090009AE024FF924D128573D2BE
:1025F7003F7BFF7A0E79EA02976F9001E2E064036E
:1026070070341279899000B4E060031279AD9000BC
:10261700B1E0900000F0E49001E2F09001E3E09077
:102627000052F09001E4E0900053F0E4900190F044
:1026370090018F022A029001E2E0602D12798990C1
:1026470000B4E060031279AD9000B1E0900000F0B3
:1026570090005BE0900052F090005374FEF0E4901D
:102667000190F090018F022AA2305B61304A5EC26E
:102677004A90004EE0FFC39415505274D22FF58252
:10268700E43400F583E0FFA248E4336F703FA248CB
:10269700924990004EE0900191F090004FE0900138
:1026A70092F090004DE0900193F01270CB9001935F
:1026B700E0641F6018900191E0FF900192E0FD7CBB
:1026C7000012860E90018F7402F0022D62C24A1228
:1026D700002EBF01171279899000B4E060031279C8
:1026E700AD9000B1E0900000F0022A909000B5E0B4
:1026F70060251294A9EF6401600612986EBF011756
:102707007BFF7A0E79FB12976F900092E078A0F624
:102717009001907409F0221294A9EF640170683057
:102727003B28C23B90019C04F0D239853E3FE53FF0
:1027370075F010A424DAF9740F35F0FA7BFF1297BD
:102747006FAF3F128BFAC239802A30413AC24190AB
:10275700019EE534F075F010A4241AF9741335F0CE
:10276700FA7BFF12976F90019EE0FF1289F79001A5
:102777009C7402F090018F7405F0E4900190F09042
:102787000092E078A0F622C23BC24178A2E6184642
:10279700703F900099E060397BFF7A0F790C1297B0
:1027A7006F900099E0FF78A1760008A60790005285
:1027B70074FFF0900053F01279899000B4E0600341
:1027C7001279AD9000B1E0900000F0900190022CDA
:1027D700F19000A4E0FF7003022D679001A6E0606E
:1027E70003022D679000A2E0FE60107003022D67C0
:1027F7009001A2E064016003022D679001A6EFF04B
:10280700E49001A2F01279899000B4E06003127994
:10281700AD9000B1E0900000F090005BE0900052B6
:10282700F090005374FDF0E4900190F090018F0454
:10283700F022900000E06003022D67305703022D5D
:102847006790005BE0FF90015BF090015C74FFF024
:1028570090015DEFF090015EF090009AE024FF9206
:102867004D128573D23F12716D9001907403F0225F
:10287700787DE66003022D67305703022D67127DCE
:10288700D0127DDF90008DE0900001F090019074F0
:1028970004F022900001E06003022D6712798F9007
:1028A70000B4E060031279B3E4900190F09001A2C4
:1028B70004F090005274FFF0900053F02230A5030B
:1028C70002298790005BE0900052F0900098E0901A
:1028D7000053F01294A9BF010512799B8003127966
:1028E700A1787DE66003022D67305703022D6790BC
:1028F7000197E07034D23F90009AE024FF924D9008
:10290700005BE0FF90015BF0900098E090015CF0C5
:1029170090015DEFF012698290015EEFF01285730E
:102927009001977402F002716D12828EEF6401704C
:102937004CD23F900158E0FF2442F582E43401F580
:1029470083E090015BF0742D2FF582E43401F58369
:10295700E090015CF0900158E090015DF012646234
:1029670090015EEFF090015BE024D2F582E4340041
:10297700F583E024FF924D128573022D46022D4602
:10298700022D62900000E06003022D6730570302BA
:102997002D67787DE66003022D6790005274FFF083
:1029A700900053F012835CEF64017053900158E07C
:1029B700FF2442F582E43401F583E090015BF07473
:1029C7002D2FF582E43401F583E090015CF090014E
:1029D70058E090015DF0129A6990015EEFF0900166
:1029E7005BE024D2F582E43400F583E024FF924DC6
:1029F700128573D23F12716D9001907407F0229087
:102A0700008DE0900001F0900190022AA2305B63F4
:102A1700304A62C24A90004EE0FFC3941550567484
:102A2700D22FF582E43400F583E0FFA248E4336F48
:102A37007043A248924990004EE0900191F09000B7
:102A47004FE0900192F090004DE0900193F01270EA
:102A5700CB900193E0641F601C900191E0FF90010F
:102A670092E0FD7C0012860EE4900190F090018FB9
:102A7700022CF1C24A787DE66003022D67305703C6
:102A8700022D6712002EEF60079001907406F02266
:102A970090008DE0900001F09001907408F0229072
:102AA7000001E06003022D6712798F9000B4E060A7
:102AB700031279B39001A27401F0E4900190F090B1
:102AC700005274FFF0900053F0027DDF305B6330FB
:102AD7004A60C24A90004EE0FFC39415505474D226
:102AE7002FF582E43400F583E0FFA248E4336F70EA
:102AF70041A248924990004EE0900191F090004F1A
:102B0700E0900192F090004DE0900193F01270CBAD
:102B1700900193E0641F601A900191E0FF90019289
:102B2700E0FD7C0012860EE4900190F090018F0288
:102B37002CF1C24A78A0E66003022D6790005BE0A3
:102B4700900052F090005374FDF09000B5E0FF64E0
:102B5700016004EFB402151294A9BF010F9000930E
:102B6700E0900005F0900190740AF0229000B5E023
:102B7700FF64036004EFB4041512986EBF010F9051
:102B87000093E0900005F0900190740BF022022D65
:102B9700621294A9BF0108900093E0900005F0909D
:102BA7000005E07003022C819000B5E0B401097BB9
:102BB700FF7A0F791D022CA01279897BFF7A0F7992
:102BC7002E1297A4787DE66003022D533057030237
:102BD7002D53900197E07031D23F90009AE024FF87
:102BE700924D90005BE0FF90015BF0900098E090C1
:102BF700015CF090015DEFF012698290015EEFF0E9
:102C0700128573900197022CF112828EEF64017086
:102C17004CD23F900158E0FF2442F582E43401F59D
:102C270083E090015BF0742D2FF582E43401F58386
:102C3700E090015CF0900158E090015DF012646251
:102C470090015EEFF090015BE024D2F582E434005E
:102C5700F583E024FF924D128573022D469001976C
:102C6700E014F0022D5312986EBF0108900093E014
:102C7700900005F0900005E0701212798F9000998E
:102C8700E0FF78A1760008A607022D629000B5E064
:102C9700B403097BFF7A0F793F0297A47BFF7A0F72
:102CA70079501297A4127989787DE66003022D5333
:102CB700305703022D53900197E07032D23F9000B6
:102CC7009AE024FF924D90005BE0FF90015BF0904B
:102CD7000098E090015CF090015DEFF0126982903E
:102CE700015EEFF01285739001977402F022128251
:102CF7008EEF64017050D23F900158E0FF2442F5F7
:102D070082E43401F583E090015BF0742D2FF582A6
:102D1700E43401F583E090015CF0900158E0900104
:102D27005DF012646290015EEFF090015BE024D2E7
:102D3700F582E43400F583E024FF924D1285739009
:102D47000197E014F022900197E014F090005BE007
:102D5700900052F090005374FDF022E4900190F03F
:012D67002249
:10897100129079900190E0FF700C900000E070750A
:1089810090019004F022EF64017029205D1D900197
:10899100C27419F0A3E4F09001BE04F0D25D90011D
:1089A1009004F07BFF7A0F796180067BFF7A0F7963
:1089B100720297A4900190E0FFB402189001E5E0E3
:1089C10064017031F090008DE0900001F090019011
:1089D1007403F022EFB40314900001E070171279D0
:1089E1008F9000B4E060051279B38000E490018FAC
:0689F100F0900190F0225D
:1087CC00900190E0703B900068E0602B12798990EA
:1087DC0000B4E060031279AD9000B1E0900000F0BD
:1087EC00900191E0900052F0900192E0900053F0D3
:1087FC009001907401F022E4900190F090018FF0C0
:10880C0022900190E06401703E205D32900191E075
:10881C00FE900192E07C002400FFEC3E9001C2F03F
:10882C00A3EFF09001BE7401F0D25D900069E0906E
:10883C00018F6004740480027403F0E4800E7BFFEB
:10884C007A0F79720297A4E490018FF0900190F066
:01885C0022F9
:1052F300900190E0704A900000E0600302565FA2C4
:1053030049924D900191E090015BF0900192E09001
:10531300015CF090005BE090015DF0126982900106
:105323005EEFF0128573D23F12716D90019774088E
:10533300F090008CE0900006F09001907401F02250
:10534300900190E06401703E127222EF600280557A
:10535300787DE6600302565F30570302565F762876
:10536300D257900197E014F0E0600302565F740295
:10537300F090008CE0900006F090008EE090000C1E
:10538300F09001908069900190E064026003025400
:1053930050127222EF6002800C90008EE0600D903C
:1053A300000CE070079001907403F022787DE660B2
:1053B3000302565F30570302565F900197E0703344
:1053C300A249924D900191E090015BF0900192E02F
:1053D30090015CF090005BE090015DF012698290B7
:1053E300015EEFF0128573D23F12716D90019774D5
:1053F30002F02212828EEF6401704F900158E0FF99
:105403002442F582E43401F583E090015BF0742DCE
:105413002FF582E43401F583E090015CF0900158AC
:10542300E090015DF012646290015EEFF090015B29
:10543300E024D2F582E43400F583E024FF924D1298
:105443008573D23F12716D0255030255039001908B
:10545300E06403702E205D229001C2F0A374FFF07C
:105463009001BE7401F0D25D127DD01279A1E49057
:105473000198F09001907404F0227BFF7A0F797207
:105483000297A4900190E064047043787DE6600382
:1054930002565F30570302565FA249924D90019125
:1054A300E090015BF0900192E090015CF090015D6F
:1054B300741FF0129A6990015EEFF01285739001E8
:1054C300977403F012716D9001907405F0229001AE
:1054D30090E0FF64057030787DE6600302565F302C
:1054E300570302565F900197E0700F90008DE09094
:1054F3000001F09001907406F022787D7628D2574F
:10550300900197E014F022EF64066003025648907E
:1055130000B5E0601F303B0930410612986EEF7012
:1055230013E490018FF0900190F0900092E078A046
:10553300F602563B305B7A304A77C24A90004EE01F
:10554300FFC39415506B74D22FF582E43400F583B6
:10555300E0FFA248E4336F7058A248924990004E8E
:10556300E0900191F090004FE0900192F090004D97
:10557300E0900193F0641F6038900191E0FFC394C1
:1055830015502E74D22FF582E43400F583E0FFA288
:1055930049E433B5071B900191E0FF900192E0FDD0
:1055A3007C0012860E90018F7402F0E4900190F05B
:1055B30022C24A787DE6705520575212835CEF640D
:1055C30001704A900158E0FF2442F582E43401F56A
:1055D30083E090015BF0742D2FF582E43401F583B1
:1055E300E090015CF0900158E090015DF01264627C
:1055F30090015EEFF090015BE024D2F582E4340089
:10560300F583E024FF924D12857312716D900001B2
:10561300E0704912798F9000B4E060031279B3907F
:10562300005274FFF0900053F09001A27401F0E473
:1056330090018FF0900190F0900099E0FF78A176AF
:105643000008A60722900190E0D39406400EE49050
:0D565300018FF0900190F078A1F608F6228A
:1046B500900190E070107BFF7A0F798312976F90CD
:1046C50001907401F022900190E06401705990000E
:1046D50000E06003024AEEA249924D900191E090FC
:1046E500015BF0900192E090015CF090005BE0903E
:1046F500015DF012698290015EEFF0128573D23F81
:1047050012716D90008CE0900006F090008EE090A4
:10471500000CF09000B8E09001A3F09001977403AD
:10472500F090019014F022900190E06402702F78CF
:104735007DE66003024AEE305703024AEE7628D240
:1047450057900197E014F0E06003024AEE12799B5E
:104755009001977402F090019004F0C24A229001F2
:1047650090E064036003024863129AE5205B0890B9
:1047750000B8E07002803F9000B8E0FF600890014B
:10478500A3E070028030305B0D304A0A9001A3EF40
:10479500F0C24A12799B1294A9EF70031279A19085
:1047A50001E5E0B40104E402488890008EE0600D64
:1047B50090000CE070079001907404F022787DE67B
:1047C5006003024AEE305703024AEE900197E0700B
:1047D50033A249924D900191E090015BF0900192D6
:1047E500E090015CF090005BE090015DF012698261
:1047F50090015EEFF0128573D23F12716D900197B3
:104805007402F02212828EEF6401704F900158E01D
:10481500FF2442F582E43401F583E090015BF074F6
:104825002D2FF582E43401F583E090015CF09001D1
:1048350058E090015DF012646290015EEFF0900126
:104845005BE024D2F582E43400F583E024FF924D49
:10485500128573D23F12716D0249190249199001EF
:1048650090E06404702E205D229001C2F0A374FFD5
:10487500F09001BE7401F0D25D127DD01279A1E4F1
:10488500900198F09001907405F0227BFF7A0F79E2
:10489500720297A4900190E064057046787DE66009
:1048A50003024AEE305703024AEEA249924D9001A7
:1048B50091E090015BF0900192E090015CF0900135
:1048C5005D741FF0129A6990015EEFF01285731204
:1048D50079A19001977403F012716D90019074069F
:1048E500F022900190E0FF64067030787DE6600369
:1048F500024AEE305703024AEE900197E0700F909E
:10490500008DE0900001F09001907407F022787D11
:104915007628D257900197E014F022EF64076003E0
:10492500024AD79000B5E0601F303B0930410612BE
:10493500986EEF7013E490018FF0900190F0900065
:1049450092E078A0F6024ACA1294A9EF64016003C6
:10495500024A3490008DE0900001F0204A03024A9B
:1049650034C24A1294A9EF64016003024A349001EB
:1049750091E0FF90004EE0FEB5071290004FE0FF7A
:10498500900192E0B50706E4900195F022EEC394FC
:10499500154003024A3490004EE0FF24D2F582E42C
:1049A5003400F583E0FEA248E4336E6003024A3426
:1049B500900195E0FE701BA2489249900194EFF09A
:1049C50090004FE0900195F090004DE0900196F039
:1049D500805D90004EE0FF6E7055A24892499001AF
:1049E50091EFF090004FE0900192F090004DE09033
:1049F5000193F0641F6038900191E0FFC394155056
:104A05002E74D22FF582E43400F583E0FFA249E449
:104A150033B5071B900191E0FF900192E0FD7C000A
:104A250012860E90018F7402F0E4900190F02278C6
:104A35007DE6706020575D12835CEF6401705590D0
:104A45000158E0FF2442F582E43401F583E090014A
:104A55005BF0742D2FF582E43401F583E090015C61
:104A6500F0900158E090015DF012646290015EEFF4
:104A7500F090015BE024D2F582E43400F583E02474
:104A8500FF924D1285739001907406F0E490018FAA
:104A9500F012716D900001E0703812798F9000B4BA
:104AA500E060031279B390005274FFF0900053F068
:104AB5009001A27401F0E490018FF0900190F01242
:104AC5007DD0127DDF900099E0FF78A1760008A6E1
:104AD5000722900190E0D39407400EE490018FF0F7
:0A4AE500900190F078A1F608F62287
:102D6800900190E06003022E4E1294A9EF64017066
:102D78005B304A58C24A90004EE0FFC39415504C4D
:102D880074D22FF582E43400F583E0FFA248E433DF
:102D98006F7039A248924990004EE0900191F090EE
:102DA800004FE0900192F090004DE0900193F012F6
:102DB80070CB900193E0641F6012900191E0FF9046
:102DC8000192E0FD7C0012860E0231B2C24A78A060
:102DD800E660030232E71294A9EF6401705690008E
:102DE8005EE0702412798F9000B4E060031279B32A
:102DF8009000B5E0B4010F90005BE0900052F090B5
:102E0800005374FEF02280381279899000B4E06093
:102E1800031279AD12799B9000B1E0900000F09018
:102E2800005BE0900052F090005374FEF090019027
:102E38007401F02212798F9000B4E060031279B324
:102E4800C239E40232E3900190E064017061305DC0
:102E580003022FAF90019CE0FBB4010FE53F240073
:102E6800FEE434159001C2F0A3CEF0EBB402119049
:102E7800019EE02400FEE434169001C2F0A3CEF0D7
:102E88009001BE7401F0D25D90008EE090000CF0CD
:102E9800900091E0900008F0900060E0600BE490F2
:102EA8000190F090018F022FD79001900232D790B5
:102EB8000190E06402707A900000E060030232E75B
:102EC80090019CE064017025AF3F1299BBE53F7506
:102ED800F010A424DAF9740F35F0FA7BFF12976F1B
:102EE800E53F75F010A424DAF9740F803590019C41
:102EF800E0640260030232E790019EE0FF121EBA0E
:102F080090019EE075F010A4241AF9741335F0FAB4
:102F18007BFF12976F90019EE075F010A4241AF9B8
:102F2800741335F0FA7BFF1297A49001907403F0A4
:102F380022900190E064037024126F6FEF600280AA
:102F48001290008EE070030232E790000CE06003FC
:102F58000232E7127DD09001907404F02290019023
:102F6800E06404704B205D3F9001C2F0A374FFF051
:102F78009001BE7401F0D25D127DDF1279A1E49058
:102F8800019DF090005DE0600E90009FE0900009C8
:102F9800F09001900232629000A0E0900002F012DE
:102FA800009690019080287BFF7A0F79720297A48F
:102FB800900190E0640560030230C2900009E0705F
:102FC800121200969000A0E0900002F09001907418
:102FD80006F0221294A9EF6401706B120096303B40
:102FE80030C23B90019C7401F0853E3FC239E53FF9
:102FF80075F010A424DAF9740F35F0FA7BFF1297F4
:103008006FAF3F128BFAE4900190F090018F02327B
:1030180062304132C24190019EE534F075F010A44F
:10302800241AF9741335F0FA7BFF12976F90019EFA
:10303800E0FF1289F790019C7402F0E4900190F08F
:1030480090018F023262C23BC2411294A9EF64011F
:103058007065304A62120096C239C24A90004EE04A
:10306800FFC39415505174D22FF582E43400F583D0
:10307800E0FFA248E4336F703EA248924990004EA8
:10308800E0900191F090004FE0900192F090004D97
:10309800E0900193F01270CB900193E0641F6017E9
:1030A800900191E0FF900192E0FD7C0012860E9065
:1030B800018F740202313FC24A22900190E06406F7
:1030C80060030231BB900002E07007900190740722
:1030D800F0221294A9EF64017062303B2BC23B903E
:1030E800019C04F0853E3FC239E53F75F010A424E9
:1030F800DAF9740F35F0FA7BFF12976FAF3F128B36
:10310800FA90018F7405802F304131C24190019EA1
:10311800E534F075F010A4241AF9741335F0FA7B2D
:10312800FF12976F90019EE0FF1289F790019C743F
:1031380002F090018F7405F0E40231F4C23BC24101
:103148001294A9EF64017068304A65120096C2397A
:10315800C24A90004EE0FFC39415505474D22FF524
:1031680082E43400F583E0FFA248E4336F7041A2A3
:1031780048924990004EE0900191F090004FE09005
:103188000192F090004DE0900193F01270CB900105
:1031980093E0641F601A900191E0FF900192E0FDB6
:1031A8007C0012860EE4900190F090018F0232D7D5
:1031B800C24A22900190E0640760030232DE900068
:1031C80001E0702D12798F9000B4E060031279B39A
:1031D800127DDF900099E0FF78A1760008A607909D
:1031E80001A27401F0C239E490018FF0900190F0CF
:1031F800221294A9EF64017065303B2CC23B900108
:103208009C04F0853E3FE53F75F010A424DAF9747C
:103218000F35F0FA7BFF12976FAF3F128BFAE490ED
:103228000190F090018F8032304133C24190019E6D
:10323800E534F075F010A4241AF9741335F0FA7B0C
:10324800FF12976F90019EE0FF1289F790019C741E
:1032580002F0E4900190F090018F7405F022C23BD7
:10326800C2411294A9EF64017069304A661200964F
:10327800C239C24A90004EE0FFC39415505574D22B
:103288002FF582E43400F583E0FFA248E4336F7041
:1032980042A248924990004EE0900191F090004F70
:1032A800E0900192F090004DE0900193F01270CB05
:1032B800900193E0641F601B900191E0FF900192E0
:1032C800E0FD7C0012860EE4900190F090018F746E
:1032D80002F022C24A22E4900190F090018FF0227D
:103D5D00900190E070127BFF7A0F799412976F901B
:103D6D0001907401F002799B900190E06401706004
:103D7D00900000E0600302424F90008EE090000C36
:103D8D00F09000B8E09001A3F090019CE0B4011216
:103D9D00AF3F1299BBE53F75F010A424DAF9740F0B
:103DAD00802090019CE06402600302424F90019ECE
:103DBD00E0FF121EBA90019EE075F010A4241AF9CE
:103DCD00741335F0FA7BFF1297A490019002423FD5
:103DDD00900190E064026003023E6D129AE5205B53
:103DED00089000B8E07002800C9000B8E0600B9075
:103DFD0001A3E070051279A1805F305B329000B8AD
:103E0D00E09001A3F090019CE0B4010D303B0AE578
:103E1D003FB53E05C23B12799B90019CE0B4020F69
:103E2D0030410C90019EE0B53405C24112799B12D0
:103E3D0094A9EF70031279A19001E5E0B401051288
:103E4D007DD0803790008EE0700302424F90000CC1
:103E5D00E0600302424F127DD09001907403F02276
:103E6D00900190E0B40324205D189001C2E4F0A30A
:103E7D0074FFF09001BE7401F0D25D900190740456
:103E8D00F0227BFF7A0F79720297A4900190E06483
:103E9D0004702C127DDF1279A1E490019DF0900049
:103EAD005DE0600E90009FE0900009F0900190029F
:103EBD0041979000A0E0900002F0120096801C90B7
:103ECD000190E064056003023FED900009E070127F
:103EDD001200969000A0E0900002F0900190740600
:103EED00F0221294A9EF64016003023F791200964B
:103EFD00303B39C23BE53F653E700302424F9001B6
:103F0D009C7401F0853E3FC239E53F75F010A42445
:103F1D00DAF9740F35F0FA7BFF12976FAF3F128B02
:103F2D00FAE4900190F090018F02419730413DC22B
:103F3D004190019EE06534700302424F90019EE571
:103F4D0034F075F010A4241AF9741335F0FA7BFFD0
:103F5D0012976F90019EE0FF1289F790019C7402F9
:103F6D00F0E4900190F090018F024197C23BC24165
:103F7D001294A9EF64017065304A62120096C2393D
:103F8D00C24A90004EE0FFC39415505174D22FF5E4
:103F9D0082E43400F583E0FFA248E4336F703EA263
:103FAD0048924990004EE0900191F090004FE090C2
:103FBD000192F090004DE0900193F01270CB9001C2
:103FCD0093E0641F6017900191E0FF900192E0FD76
:103FDD007C0012860E90018F7402024087C24A2225
:103FED00900190E064066003024103900002E070CE
:103FFD000F90008DE0900001F09001907407F02279
:10400D001294A9EF64017077303B35C23BE53F65F3
:10401D003E700302424F90019C7401F0853E3FC2F9
:10402D0039E53F75F010A424DAF9740F35F0FA7BF9
:10403D00FF12976FAF3F128BFA90018F7405803A84
:10404D0030413CC24190019EE06534700302424F05
:10405D0090019EE534F075F010A4241AF97413350F
:10406D00F0FA7BFF12976F90019EE0FF1289F79097
:10407D00019C7402F090018F7405F0E40241CDC2F1
:10408D003BC2411294A9EF64017068304A65120079
:10409D0096C239C24A90004EE0FFC3941550547435
:1040AD00D22FF582E43400F583E0FFA248E4336FAC
:1040BD007041A248924990004EE0900191F090001D
:1040CD004FE0900192F090004DE0900193F012704E
:1040DD00CB900193E0641F601A900191E0FF900175
:1040ED0092E0FD7C0012860EE4900190F090018F1D
:1040FD0002423FC24A22900190E0640760030242EF
:10410D00461294A9EF6401600302419B90008DE07B
:10411D00900001F0303B36C23BE53F653E70030237
:10412D00424F90019C7401F0853E3FE53F75F010C4
:10413D00A424DAF9740F35F0FA7BFF12976FAF3FB5
:10414D00128BFAE4900190F090018F803D30413E4A
:10415D00C24190019EE06534700302424F90019E72
:10416D00E534F075F010A4241AF9741335F0FA7BC8
:10417D00FF12976F90019EE0FF1289F790019C74DA
:10418D0002F0E4900190F090018F7405F022C23B93
:10419D00C241900001E0702D12798F9000B4E06063
:1041AD00031279B3127DDF900099E0FF78A17600BC
:1041BD0008A6079001A27401F0C239E490018FF0B6
:1041CD00900190F0221294A9EF64017069304A6653
:1041DD00120096C239C24A90004EE0FFC3941550AA
:1041ED005574D22FF582E43400F583E0FFA248E444
:1041FD00336F7042A248924990004EE0900191F0C9
:10420D0090004FE0900192F090004DE0900193F0FE
:10421D001270CB900193E0641F601B900191E0FF41
:10422D00900192E0FD7C0012860EE4900190F090DA
:10423D00018F7402F022C24A22E4900190F09001A5
:03424D008FF022CD
:104F0000900190E070469001E3E0900052F0900133
:104F1000E4E0900053F07BFF7A0F79A512976FE4DD
:104F20009001E2F0900052E0FF900053E0FD7C0021
:104F300012860E900052E024D2F582E43400F5830C
:104F4000E024FF92499001907401F022900190E0DA
:104F50006401704B900000E060030252F2A249929B
:104F60004D9001E3E090015BF09001E4E090015C82
:104F7000F090005BE090015DF012698290015EEFBD
:104F8000F0128573D23F12716D900082E09001A4FF
:104F9000F090008EE090000CF09001900252E290B0
:104FA0000190E0640260030250A0129AE5305B10A9
:104FB000304A0D900082E09001A4F0C24A12799B21
:104FC0001294A9EF70031279A19001E5E0B4010CED
:104FD000E4F0127DD09001907404F0229001A4E0DE
:104FE0007008900082E06002800C90008EE06010FB
:104FF00090000CE0700A127DD09001907403F022B2
:10500000787DE660030252F23057030252F29001BB
:1050100097E07032A249924D9001E3E090015BF07D
:105020009001E4E090015CF090005BE090015DF0A5
:1050300012698290015EEFF0128573D23F12716D9A
:105040009001970252E212828EEF6401704F90013C
:1050500058E0FF2442F582E43401F583E090015BDF
:10506000F0742D2FF582E43401F583E090015CF0BB
:10507000900158E090015DF012646290015EEFF0E3
:1050800090015BE024D2F582E43400F583E024FF54
:10509000924D128573D23F12716D02514D02514DE6
:1050A000900190E0B40323205D179001C2E4F0A3C7
:1050B00074FFF09001BE7401F0D25D900190740411
:1050C000F07BFF7A0F79720297A4900190E064045C
:1050D0007049127DDF1279A1787DE660030252F2F9
:1050E0003057030252F2A249924D900191E0900193
:1050F0005BF0900192E090015CF090015D741FF014
:10510000129A6990015EEFF0128573900197740313
:10511000F012716D9001907405F022900190E0FF03
:1051200064057030787DE660030252F23057030266
:1051300052F2900197E0700F90008DE0900001F026
:105140009001907406F022787D7628D257900197CE
:10515000E014F022EF640660030252E9900001E0DF
:10516000702A12798F9000B4E060031279B3127D37
:10517000DF900099E0FF78A1760008A6079001A2D1
:105180007401F0C239E490018FF080691294A9EFA4
:1051900064017066303B2DC23B90019C04F0853E5B
:1051A0003FC239E53F75F010A424DAF9740F35F0E9
:1051B000FA7BFF12976FAF3F128BFA90018F740545
:1051C000F0E48031304133C24190019EE534F07506
:1051D000F010A4241AF9741335F0FA7BFF12976FBC
:1051E00090019EE0FF1289F790019C7402F09001FB
:1051F0008F7405F0E4900190F022C23BC2411294FA
:10520000A9EF640160030252E690008DE090000176
:10521000F0204A030252E6120096C239C24A9001B7
:1052200091E0FF90004EE0FEB5071290004FE0FFC6
:10523000900192E0B50706E4900195F022EEC39448
:105240001540030252E690004EE0FF24D2F582E4BE
:105250003400F583E0FEA248E4336E60030252E6B8
:10526000900195E0FE701BA2489249900194EFF0E6
:1052700090004FE0900195F090004DE0900196F085
:10528000806490004EE0FF6E705CA24892499001ED
:1052900091EFF090004FE0900192F090004DE0907F
:1052A0000193F01270CB900193E0641F603890017D
:1052B00091E0FFC39415502E74D22FF582E4340090
:1052C000F583E0FFA249E433B5071B900191E0FFAD
:1052D000900192E0FD7C0012860EE4900190F09027
:1052E000018F7402F022C24A22E4900190F09001F2
:0352F0008FF0221A
:10385000900190E0706390005BE0900052F0900067
:103860005374FEF09001E2E0B4011D9001E4E0F534
:103870003F7BFF7A0F79B612976F9001E4E0FF1259
:103880008BFA90019C7401F09001E2E0B4021F9069
:1038900001E4E090019EF07BFF7A0F79C912976FE7
:1038A0009001E4E0FF1289F790019C7402F0E4902B
:1038B00001E2F090019004F022900190E064017028
:1038C00058900000E06003023D5C90008EE09000A4
:1038D0000CF090019CE0B40112AF3F1299BBE53FA0
:1038E00075F010A424DAF9740F802090019CE06434
:1038F000026003023D5C90019EE0FF121EBA90013F
:103900009EE075F010A4241AF9741335F0FA7BFFC9
:103910001297A4900190023D4C900190E0640270D7
:1039200061129AE5305B2A90019CE0B4010D303BB6
:103930000AE53FB53E05C23B12799B90019CE0B47D
:10394000020F30410C90019EE0B53405C24112795E
:103950009B1294A9EF70031279A19001E5E0B401E4
:1039600005127DD0803790008EE07003023D5C90A0
:10397000000CE06003023D5C127DD0900190740366
:10398000F022900190E0B40324205D189001C2E47D
:10399000F0A374FFF09001BE7401F0D25D9001902D
:1039A0007404F0227BFF7A0F79720297A490019041
:1039B000E064047027127DDF1279A190005DE06061
:1039C0000E90009FE0900009F0900190023CD7908B
:1039D00000A0E0900002F0120096801C900190E0A0
:1039E00064056003023AFD900009E070121200962F
:1039F0009000A0E0900002F09001907406F0221276
:103A000094A9EF64016003023A89120096303B39B1
:103A1000C23BE53F653E7003023D5C90019C740132
:103A2000F0853E3FC239E53F75F010A424DAF97401
:103A30000F35F0FA7BFF12976FAF3F128BFAE490CD
:103A40000190F090018F023CD730413DC24190017E
:103A50009EE065347003023D5C90019EE534F07594
:103A6000F010A4241AF9741335F0FA7BFF12976F43
:103A700090019EE0FF1289F790019C7402F0E4909F
:103A80000190F090018F023CD7C23BC2411294A931
:103A9000EF64017065304A62120096C239C24A90E2
:103AA000004EE0FFC39415505174D22FF582E434D8
:103AB00000F583E0FFA248E4336F703EA2489249CC
:103AC00090004EE0900191F090004FE0900192F054
:103AD00090004DE0900193F01270CB900193E06460
:103AE0001F6017900191E0FF900192E0FD7C0012B1
:103AF000860E90018F7402023B97C24A2290019079
:103B0000E064066003023C13900002E0700F900036
:103B10008DE0900001F09001907407F0221294A9BA
:103B2000EF64017077303B35C23BE53F653E700383
:103B3000023D5C90019C7401F0853E3FC239E53F37
:103B400075F010A424DAF9740F35F0FA7BFF1297A0
:103B50006FAF3F128BFA90018F7405803A30413C71
:103B6000C24190019EE065347003023D5C90019E6D
:103B7000E534F075F010A4241AF9741335F0FA7BCB
:103B8000FF12976F90019EE0FF1289F790019C74DD
:103B900002F090018F7405F0E4023C49C23BC2413F
:103BA0001294A9EF64017068304A65120096C23918
:103BB000C24A90004EE0FFC39415505474D22FF5C2
:103BC00082E43400F583E0FFA248E4336F7041A241
:103BD00048924990004EE0900191F090004FE090A3
:103BE0000192F090004DE0900193F01270CB9001A3
:103BF00093E0641F601A900191E0FF900192E0FD54
:103C00007C0012860EE4900190F090018F023D4CF2
:103C1000C24A22900190E064076003023D53900085
:103C200001E0702A12798F9000B4E060031279B33A
:103C3000900099E0FF78A1760008A6079001A27491
:103C400001F0C239E490018FF0900190F0221294BB
:103C5000A9EF64016003023CDB90008DE09000015D
:103C6000F0303B36C23BE53F653E7003023D5C9061
:103C7000019C7401F0853E3FE53F75F010A424DA05
:103C8000F9740F35F0FA7BFF12976FAF3F128BFA82
:103C9000E4900190F090018F803D30413EC2419010
:103CA000019EE065347003023D5C90019EE534F0B6
:103CB00075F010A4241AF9741335F0FA7BFF1297EB
:103CC0006F90019EE0FF1289F790019C7402F0E46E
:103CD000900190F090018F7405F022C23BC2411216
:103CE00094A9EF64017069304A66120096C239C225
:103CF0004A90004EE0FFC39415505574D22FF582C0
:103D0000E43400F583E0FFA248E4336F7042A24838
:103D1000924990004EE0900191F090004FE09001A8
:103D200092F090004DE0900193F01270CB900193CF
:103D3000E0641F601B900191E0FF900192E0FD7C28
:103D40000012860EE4900190F090018F7402F02230
:0D3D5000C24A22E4900190F090018FF02211
:1000A600202020202020202020202020202020204A
:1000B6005245504541544552204E554D42455220D9
:1000C6002020202020202020203120746F20323054
:1000D600202053495445204E554D4245522020205C
:1000E6002020202020202020203120746F20393924
:1000F6008202001101021501148202011103041586
:1001060001632020202020202020202020202020C5
:1001160020202020202020202020202020202020D9
:10012600202020434F5552544553592042454550AF
:100136002020204354435353204F4E2048414E47DE
:10014600202020205553455220454E41424C452003
:10015600202020205245534552564520544F4E45A7
:10016600202020204E4554574F524B204D4F44459A
:100176002020204E4554574F524B204E554D424558
:100186005220202020202020202020202020202037
:100196002020202020202020202020202020202059
:1001A6002020202020202020202020202020202049
:1001B6002020202020202020202020202020202039
:1001C6002020202020202020202020202020313DFB
:1001D600454E2020202020202020202020204D4F6A
:1001E6004445202020202020202020202020544F5D
:1001F6004E4564010011020C150001640200110352
:100206000C15000164040011040C150001640800BB
:1002160011050C15000164100011060D150002C829
:10022600030111070A190101202020202020202087
:1002360020202020202020202020202020202020B8
:10024600202020202020202020434F555254455363
:100256005920424545502020204354435353204FB4
:100266004E2048414E4720202020555345522045D8
:100276004E41424C4520202020205245534552569F
:100286004520544F4E45202020204E4554574F526E
:100296004B204D4F44452020204E4554574F524B3E
:1002A600204E554D4245522020202020202020203F
:1002B6002020202020202020202020202020202038
:1002C6002020202020202020202020202020202028
:1002D6002020202020202020202020202020202018
:1002E6002020202020202020202020202020202008
:1002F60020202020313D454E202020202020202077
:10030600202020204D4F4445202020202020202042
:1003160020202020544F4E4564010011020C150088
:100326000164020011030C15000164040011040CA1
:1003360015000164080011050C1500016410001178
:10034600060D150001C8030111070A190101202035
:100356002020202020202020202020202020202097
:100366002020202020202020202020202020204364
:100376004F55525445535920424545502020202080
:100386005553455220454E41424C4520202020439E
:10039600524F535320544F4E45204D4F4445204312
:1003A600544353532F4443532043524F5353202017
:1003B6004E4554574F524B204D4F44452020204E1A
:1003C6004554574F524B204E554D42455220202002
:1003D6002020202020202020202020202020202017
:1003E60020202020202020202020313D454E202086
:1003F600202020202020202020204D4F4445202052
:1004060020202020202020202020544F4E45202030
:1004160020202020202020202020202020206401B1
:1004260000110209150001640200110309150001FB
:1004360064040011060A150001C8030111070C190E
:1004460001012020202020202020202020202020E4
:100456002020202020202020202020202020202096
:10046600202001010101010101010100000000003D
:100476000000000000000000000000000000000076
:100486000000000000000000000000000000000066
:100496000000000000000000000000000000000056
:1004A6000000000000000000000000000000000046
:1004B60000000000000000000000000020202020B6
:1004C6002020202020202020202020202020202026
:1004D6002020202020202020202020200101010192
:1004E6000101010101000000000000000000000001
:1004F60000000000000000000000000000000000F6
:1005060000000000000000000000000000000000E5
:1005160000000000000000000000000000000000D5
:1005260000000000000000000000000000000000C5
:100536000000000000002020202020202020202075
:1005460020202020202020202020202020202020A5
:1005560020202020202001010101010101010120AC
:100566002020202020202020202020202020202085
:100576002020202020202020202020202020202075
:1005860054454C434F2050524F4752414D20202056
:10059600524144494F2050524F4752414D2020204E
:1005A60050484F4E452050524F4752414D20202033
:1005B600434F4D50552050524F4752414D20202019
:1005C6002041434345535320434F44452020204474
:1005D600544D462054454C434F204C4556454C44BB
:1005E600544D4620524144494F204C4556454C42B5
:1005F60045455020524144494F204C4556454C42B2
:100606004545502054454C434F204C4556454C4398
:1006160057494420524144494F204C4556454C5673
:100626004F49434520524144494F204C45564C566C
:100636004F4943452054454C434F204C45564C505A
:1006460041474520524144494F204C4556454C436D
:100656005443535320524144494F204C45564C4431
:10066600435320524144494F204C4556454C204C5B
:10067600545220524144494F204C4556454C205235
:10068600505420524144494F204C4556454C205425
:10069600454C434F20524144494F204C45564C52FD
:1006A6004144494F2054454C434F204C45564C52EB
:1006B6004144494F204C494D4954204C45564C2005
:1006C600434F53204F5220535155454C4348202009
:1006D60020434F5320504F4C4152495459202043F8
:1006E6004F53205452494747455220564F4C544386
:1006F6004F5320414351554953542054494D454386
:100706004F532052454C454153452054494D4520B1
:1007160053454E534520504F4C415249545920534E
:10072600454E205452494747455220564F4C545344
:10073600454E20414351554953542054494D455344
:10074600454E2052454C454153452054494D452080
:100756004C545220484F4C442044454C415920505B
:100766005454205455524E4F46462054494D4552F6
:10077600455045415445522054494D454F55542006
:1007860020414E54492D4B45524348554E4B20204F
:1007960020535155454C4348205441494C20202074
:1007A60043544353532F44435320484F4C44204310
:1007B600524F535320425553592044454C415943B7
:1007C600524F5353204255535920484F4C442020F2
:1007D600204C54522053594E432042495420202045
:1007E600414456414E43454420204C4F434B202024
:1007F60020202020202020202020202020202020F3
:1008060020202020202020202020202020202020E2
:1008160020202020202020202020202020202020D2
:1008260020202020202020202020202020202020C2
:100836002020202020202020202020313D454E2031
:1008460020202020202020202020524154494F20C3
:1008560020202020202020202020303D434F5320E0
:1008660020202020202020202020313D504F5320C2
:10087600202020202020202020202031204D532001
:10088600202020202020202020203130204D5320E1
:10089600202020202020202020313030204D5320C1
:1008A60020202020202020202020202053454320C7
:1008B600202020202020202020313D534B4950204D
:1008C6002020202020202020202020202020202022
:1008D6002020202020202020202020202020202012
:1008E6005052494F52495459204C4556454C2020A8
:1008F6004C545220454E434F444520504F4C2020E7
:100906004C5452204445434F444520504F4C2020E0
:10091600205445535420494420434F444520204900
:10092600444C45204D45535341474520544D522094
:100936002020204152454120424954202020202099
:100946004D4153544552204F5220534C4156452059
:1009560044435320454E434F444520504F4C20209E
:10096600444353204445434F444520504F4C202098
:10097600434F5552544553592044454C4159202024
:10098600202048414E472054494D452020202043F1
:100996004152524945522044524F5020444C59200E
:1009A600204143434553532044454C41592020534D
:1009B600544154494F4E204944204D4F4445202030
:1009C600564F494345204F52204357494420202043
:1009D60020494420494E54455256414C202020205F
:1009E6002020435749442053504545442020202089
:1009F60043574944204652455155454E43592020B8
:100A06002043574944204D45535341474520202014
:100A16005455524E5F4F4E2044454C41592020209C
:100A26005455524E5F4F46462044454C415920206E
:100A360042454550204652455155454E4359205250
:100A4600455045415445522044495341424C452066
:100A56004155582052454C4159204D4F4445202080
:100A660043524F53532042555359204D4F4445202E
:100A76005245504541544552204741494E20202079
:100A86002054454C434F204741494E202020204EBC
:100A96004554574F524B2048414E4754494D4520E7
:100AA6002020202020202020204C4556454C202068
:100AB600202020202020202020303D4E4F524D2047
:100AC6002020202020202020202020434F44452085
:100AD6002020202020202020202020415245412077
:100AE60020202020202020303D4D415354455220C7
:100AF600202020202020202020202031204D53207F
:100B0600202020202020202020203130204D53205E
:100B1600202020202020202020313030204D53203E
:100B26002020202020202020203130205345432023
:100B36002020202020202020202031204D494E201A
:100B460020202020202020202020204D4F444520FA
:100B56002020202020202020303D564F494345208C
:100B660020202020202020202020204652455120D1
:100B76002020202020202020202020313D454E20EE
:100B860020414C41524D20434F554E5420202020A9
:100B9600524553544F524520434F554E5420202022
:100BA6002020494E54455256414C202020202020DA
:100BB6004E4554574F524B20434F44452020204921
:100BC6004E544552434F4E4E454354204D4F444E8E
:100BD6004554574F524B20494E414354495645823E
:100BE600010011022D15000182010111032D1500CE
:100BF6000182010211042D15000182010311052D48
:100C060015000178060411060119010182030A1173
:100C1600072E1500FF82030B11082E1500FF820315
:100C26000C11092E1500FF82030D110A2E1500FF67
:100C360082030E110B2E1500FF82030F110C2E15C9
:100C460000FF820310110D2E1500FF820311110EF5
:100C56002E1500FF820312110F2E1500FF820313BB
:100C660011102E1500FF82031411112E1500FF829C
:100C7600031511122E1500FF82031611132E1500EF
:100C8600FF82031711142E1500FF82031811152E6B
:100C96001500FF82011911162F15000182011A1184
:100CA600173015000182031B11182E1500FF820252
:100CB6001C11193115006382021D111A32150063C9
:100CC60082011E111B3015000182031F111C2E15F7
:100CD60000FF820220111D31150063820221111EC0
:100CE60032150063820222111F3315026382032329
:100CF6001120321501FF8203241121341502FF82CF
:100D060002251122331500638202261123321500B3
:100D160063820227112433150363820228112532C8
:100D26001500638203291126331500FA82012A1160
:100D3600273515000182012B11385415010982014E
:100D46002C11395515000182012D113A5515000156
:100D560082032E113B561501FA82032F113C5C15B6
:100D660000FF820130113D57150001820131113E0D
:100D760058150001820132113F55160001820133D8
:100D860011405515000182023411415A1500638243
:100D9600023511425B15006382023611435A150073
:100DA6006382023711445A15006382013811455E89
:100DB60015000182013911465F15000182023A11C0
:100DC600475D15006382023B114859150463820290
:100DD6003C114960150114BE0A3D114A5611000026
:100DE600820247114B5A150063820248114D601565
:100DF6000114820149114E5E15000282014A114F0B
:100E06006115000182014B11505E15000482014CF0
:100E160011515415010982014D11525415010982CF
:100E2600024E11533415006382014F116201150001
:100E36000982015011630115000982025111645D96
:100E4600150163C803521165011501018201541190
:100E5600665E1500028203551167341500FF010115
:100E66000200000200000200000000000001010173
:100E76003132333435361432320532FFFFFF191959
:100E8600196464C8FF000180000A0180000A1E1A66
:100E9600B400001E1E1E0001000002010001000039
:100EA6000A1E630A000100050520202020202020BC
:100EB6002020200A050000000101140000010000A6
:020EC60000002A
:10976F008B758A7689777F01127DB6E49000E7F0DA
:10977F009000E7E0FFC39410501AAB75AA76A97753
:10978F008F827583001284E6FF127D879000E7E0D9
:05979F0004F080DC2253
:1097A4008B758A7689777F11127DB6E49000E7F095
:1097B4009000E7E0FFC39410501AAB75AA76A9771E
:1097C4008F827583001284E6FF127D879000E7E0A4
:0597D40004F080DC221E
:104AEF00E49001A8F0A3F09001AAF09000EBF0A3DE
:104AFF00F09000ECE02400F582E43404F583E4F058
:104B0F009000ECE004F070069000EBE004F09000F1
:104B1F00EBE07004A3E0648070D7E49000E7F090BE
:104B2F0000E7E0FFC394024003024BC0EF900E6416
:104B3F0093FF9001AAE0FE04F074002EF582E43496
:104B4F0004F583EFF09001AAE06480705B9001A8F8
:104B5F00E0FEA3E07807C333CE33CED8F9FF7C0451
:104B6F007D0012740EE49000EBF0A3F09000ECE0E7
:104B7F002400F582E43404F583E4F09000ECE004C3
:104B8F00F070069000EBE004F09000EBE07004A3EF
:104B9F00E0648070D7E49001AAF09001A9E004F0DE
:104BAF0070069001A8E004F09000E7E004F0024BDB
:104BBF002EE49000EAF0E49000E8F0A3F0E4900017
:104BCF00E7F09000E7E0FFC394034003024C63EF6C
:104BDF00900E6693FF9001AAE0FE04F074002EF58C
:104BEF0082E43404F583EFF09001AAE06480705BF7
:104BFF009001A8E0FEA3E07807C333CE33CED8F9F7
:104C0F00FF7C047D0012740EE49000EBF0A3F09093
:104C1F0000ECE02400F582E43404F583E4F0900026
:104C2F00ECE004F070069000EBE004F09000EBE095
:104C3F007004A3E0648070D7E49001AAF09001A9FA
:104C4F00E004F070069001A8E004F09000E7E004A3
:104C5F00F0024BD19000E9E004F070069000E8E01C
:104C6F0004F0C39000E9E094339000E8E094005022
:104C7F0003024BCC9000EAE004F0E0C3941450031D
:104C8F00024BC5E49000EAF0E49000E8F0A3F0E4F2
:104C9F009000E7F09000E7E0FFC394034003024D5C
:104CAF0035EF900E6993FF9001AAE0FE04F07400B7
:104CBF002EF582E43404F583EFF09001AAE06480CE
:104CCF00705B9001A8E0FEA3E07807C333CE33CE2C
:104CDF00D8F9FF7C047D0012740EE49000EBF0A372
:104CEF00F09000ECE02400F582E43404F583E4F066
:104CFF009000ECE004F070069000EBE004F0900000
:104D0F00EBE07004A3E0648070D7E49001AAF09008
:104D1F0001A9E004F070069001A8E004F09000E70C
:104D2F00E004F0024CA39000E9E004F0700690005C
:104D3F00E8E004F0C39000E9E094709000E8E0949C
:104D4F00005003024C9E9000EAE004F0E0C394147C
:104D5F005003024C97E49000E8F0A3F0E49000E7D2
:104D6F00F09000E7E0FFC394034003024E02EF9080
:104D7F000E6C93FF9001AAE0FE04F074002EF582F2
:104D8F00E43404F583EFF09001AAE06480705B9047
:104D9F0001A8E0FEA3E07807C333CE33CED8F9FFE6
:104DAF007C047D0012740EE49000EBF0A3F09000F1
:104DBF00ECE02400F582E43404F583E4F09000EC99
:104DCF00E004F070069000EBE004F09000EBE07070
:104DDF0004A3E0648070D7E49001AAF09001A9E0E9
:104DEF0004F070069001A8E004F09000E7E004F0F2
:104DFF00024D709000E9E004F070069000E8E004C6
:104E0F00F0C39000E9E094889000E8E09413500319
:104E1F00024D6B8000E49000E8F0A3F0E49000E70F
:104E2F00F09000E7E0FFC394564003024EC2EF90AC
:104E3F000E7293FF9001AAE0FE04F074002EF5822B
:104E4F00E43404F583EFF09001AAE06480705B9086
:104E5F0001A8E0FEA3E07807C333CE33CED8F9FF25
:104E6F007C047D0012740EE49000EBF0A3F0900030
:104E7F00ECE02400F582E43404F583E4F09000ECD8
:104E8F00E004F070069000EBE004F09000EBE070AF
:104E9F0004A3E0648070D7E49001AAF09001A9E028
:104EAF0004F070069001A8E004F09000E7E004F031
:104EBF00024E309000E9E004F070069000E8E00444
:104ECF00F0C39000E9E094149000E8E094005003E0
:104EDF00024E2B9001A8E0FEA3E07807C333CE3338
:104EEF00CED8F9FF7C047D0012740E127DD0027DA6
:014EFF00DFD3
:109AA200E4900059F0A3F0FFFE1273B790005BEF51
:029AB200F022A0
:1087390075530175540075556AE49001F6F0A3F07C
:108749009001F6E0FAA3E0FBC39456EA9400504086
:1087590090005BE075F056A42478FFE5F03460CF13
:108769002BCF3AFE900059F0A3EFF01273B7AB5339
:108779000555E555AA547002055414F9EF128513ED
:108789009001F7E004F070B89001F6E004F080B0D1
:1087990090009BE07004D2588002C258900097E084
:1087A90024FF924F900096E024FF924490009DE0B0
:1087B90024FF924E90009CE024FF924590007CE0BB
:0287C900F52D8C
:0187CB00228B
:108FC1007553017554007555BFE49001F6F0A3F097
:108FD1009001F6E0FEA3E0FFC39414EE9400503B31
:108FE1007C007D56128525EF24F9FFEE3460FE905A
:108FF1000059F0A3EFF01273B7AB530555E555AA2D
:10900100547002055414F9EF1285139001F7E0042E
:0B901100F070BD9001F6E004F080B5A7
:01901C002231
:10901D007553017554007555D3E49001F6F0A3F026
:10902D009001F6E0FEA3E0FFC39414EE9400503BD4
:10903D007C007D56128525EF24FEFFEE3460FE90F8
:10904D000059F0A3EFF01273B7AB530555E555AAD0
:10905D00547002055414F9EF1285139001F7E004D2
:0B906D00F070BD9001F6E004F080B54B
:0190780022D5
:108BFA008F75E49000E7F09000E7E0FBC394035020
:108C0A003E90005BE075F099A42469FDE5F034FF1D
:108C1A00FCE57575F003A42DFFE5F03CFEEB7C0046
:108C2A002FFFEC3EFE1273B79000E7E02461F58255
:108C3A00E43400F583EFF09000E7E004F080B890A8
:108C4A000061E0FE540190005CF0EE540290005D79
:108C5A00F0900061E0540490005EF0EE5408900039
:0D8C6A005FF0900061E05410900060F02277
:1089F7008F75E49000E7F09000E7E0FBC394035025
:108A07004490005BE0FF7E007C017D50128525EFDE
:108A170024A6FDEE340AFCE57575F003A42DFFE5E9
:108A2700F03CFEEB7C002FFFEC3EFE1273B790008C
:108A3700E7E02461F582E43400F583EFF09000E786
:108A4700E004F080B2900061E0FE540190005CF019
:108A5700EE540290005DF0900061E0540490005ED7
:108A6700F0EE540890005FF0900061E05410900021
:038A770060F0228A
:06860E008F758C768D775C
:10861400E49001F6F0A3F0E57724FFFFE57634FF5C
:10862400FE7C007D03128525AA06AB07AE75E575B1
:1086340025E0CE75F0EEA4FFE5F02EFEEF2448FF12
:10864400EE3423CF2BCF3AFE9001F7E02FFF9001B9
:10865400F6E03EFE1273B79001F7E02461F582E480
:108664003400F583EFF09001F7E004F07006900118
:10867400F6E004F0C39001F7E094039001F6E0946F
:10868400004094900061E0FE5401900067F0EE54C5
:0F86940002900068F0900061E05404900069F0DB
:0186A30022B4
:10997C002020202020534C41564520202020202000
:10998C0020202020204D41535445522020202020BF
:0E9AF500127CE4127DD0127DDF7F01027DB66F
:1097D9009000037414F0127DD0900003E070FA90A9
:1097E900009BE07BFF60067A99797C80047A9979FD
:1097F9008C1297A49000037414F0127DD09000038A
:04980900E070FA22EF
:10772A00C0D0C0E0C0F0C000A88475840FE55854EA
:10773A0007B4000D85E8F0A2F09220A2F192218010
:10774A0076B4010D85E8F0A2F09222A2F19223808C
:10775A0066B4020D85E8F0A2F09224A2F192258087
:10776A0056B4030D85E8F0A2F09226A2F192278082
:10777A0046B4040D85E8F0A2F09218A2F19219809D
:10778A0036B4050D85E8F0A2F0921AA2F1921B8098
:10779A0026B4060D85E8F0A2F0921CA2F1921D8093
:1077AA001685E8F0A2F0921EA2F1921F7558FF8585
:1077BA00231E85241FD260055875590A8884D00073
:1077CA00D0F0D0E0D0D032205F0122D2B7E55A54AF
:1077DA0007B4000AA22F92F7A22E92F6805EB40195
:1077EA000AA22D92F7A22C92F68051B4020AA22B79
:1077FA0092F7A22A92F68044B4030AA22992F7A227
:10780A002892F68037B4040AA23792F7A23692F683
:10781A00802AB4050AA23592F7A23492F6801DB4E2
:10782A00060AA23392F7A23292F68010B40721A276
:10783A003192F7A23092F6C25F755AFF055A7584E3
:10784A000F85E8E0A2F692E6A2F792E7F5E8C2B75A
:01785A00220B
:108F61009001D2E0FFEF12854D8F8F008F93018F1B
:108F710097028F9B038F9F048FA3058FA7068FAB4B
:108F8100078FAF088FB3098FB70A00008FBB128D0F
:108F91005F221286A42212917D22128C7722127FE7
:108FA100ED2212841D22127DEE221295A62212922A
:108FB1007522125EF6221260CF229001D2E4F022D5
:108D5F003061669001D3E4F0C261E55612854D8D06
:108D6F008D478D94488D9B498DA24A8DA94B8DB00F
:108D7F004C8DB74D8DBE4E8DC24F00008DC89001EA
:108D8F00D27401F0229001D27402F0229001D274B9
:108D9F0003F0229001D27404F0229001D27405F0F6
:108DAF00229001D27406F0229001D27407F02212A1
:0A8DBF009A3E229001D27408F022BF
:1086A4009001D3E0FFEF70189001DA7401F09001AB
:1086B400DB7401F09001D27409F09001D3E4F0224C
:1086C4009001D3E0FFEFB401189001DA7401F09047
:1086D40001DB7402F09001D2740AF09001D3E4F04B
:1086E400229001D3E0FFEF640270499001D8E4F0D6
:1086F400A3E4F09001D8E475F001128537AFF0FEE1
:10870400EF4E60269001D4E475F001128537AFF086
:10871400FE9001D8E0FCA3E0FD74002DF5827408FE
:108724003CF583E0FD12737680C97F0112008690C8
:0587340001D2E4F02277
:10917D009001D3E0FFEF70189001DA7402F09001C6
:10918D00DB7401F09001D27409F09001D3E4F02268
:10919D009001D3E0FFEFB401189001DA7402F09062
:1091AD0001DB7402F09001D2740AF09001D3E4F067
:1091BD00229001D3E0FFEFB4020A7F0112008690E6
:0591CD0001D2E4F022D4
:108C77009001D3E0FFEF70189001DA7403F09001D0
:108C8700DB7401F09001D27409F09001D3E4F02273
:108C97009001D3E0FFEFB401189001DA7403F0906C
:108CA70001DB7402F09001D27409F09001D3E4F073
:108CB700229001D3E0FFEFB4021C205F2F9001D474
:108CC700E0FEA3E0FF9001C2EEF0A3EFF0D25F90C9
:108CD70001D3E004F0229001D3E0FFEFB4030D20AD
:0D8CE7005F0A7F011200869001D2E4F022A6
:107FED009001D3E0FFEF70189001DA7404F0900166
:107FFD00DB7401F09001D27409F09001D3E4F0220A
:10800D009001D3E0FFEF640170749001D6E0FEA300
:10801D00E0FF9001D8EEF0A3EFF09001E0E4F0A3C3
:10802D00E4F09001D8E4F0A3E4F09001D8E475F009
:10803D0001128537AFF0FEEF4E602B9001D4E47541
:10804D00F001128537AFF0FE1273B79001E0E475C1
:10805D00F001128537ADF0FC74002DF58274083CEB
:10806D00F583EFF080C4900800E0FF1200869001C8
:10807D00E0E4F0A37401F09001D3E004F02290014C
:10808D00D3E0FFEF6402703F30624D9001E0E47584
:10809D00F001128537AFF0FE74002FF58274083EA3
:1080AD00F583E0FF1200869001D6E0FEA3E0FF907D
:1080BD0001E0E0FCA3E0FDC3ED9FEC9E5002222207
:1080CD009001D3E004F0229001D3E0FFEFB4030858
:0980DD003062059001D2E4F022AA
:10841D009001D3E0FFEF70189001DA7405F0900130
:10842D00DB7401F09001D27409F09001D3E4F022D5
:10843D009001D3E0FFEFB4012C9001D6E0FEA3E054
:10844D00FF128B7B900800E0FF1200869001D6741E
:10845D0004F0A3E4F09001E0E4F0A37401F09001C6
:10846D00D3E004F0229001D3E0FFEF6402703F30BF
:10847D00624D9001E0E475F001128537AFF0FE74A6
:10848D00002FF58274083EF583E0FF1200869001FF
:10849D00D6E0FEA3E0FF9001E0E0FCA3E0FDC3ED1C
:1084AD009FEC9E500222229001D3E004F022900115
:1084BD00D3E0FFEFB403083062059001D2E4F0225F
:107DEE009001D3E0FFEF70189001DA7406F0900165
:107DFE00DB7401F09001D27409F09001D3E4F0220B
:107E0E009001D3E0FFEFB401289001C27430F0A3CB
:107E1E00E4F09001D4E0FEA3E0FF9001C4EEF0A3E5
:107E2E00EFF09001BE7402F0D25F9001D3E004F047
:107E3E00229001D3E0FFEFB4020D305F03027EEF1C
:107E4E009001D3E004F0229001D3E0FFEFB4030DD4
:107E5E00205E03027EEF9001D3E004F0229001D366
:107E6E00E0FFEFB40421900800E0FF1200869001BD
:107E7E00D67404F0A3E4F09001E0E4F0A37401F0F2
:107E8E009001D3E004F0229001D3E0FFEF6405707F
:107E9E003F30624D9001E0E475F001128537AFF08E
:107EAE00FE74002FF58274083EF583E0FF12008603
:107EBE009001D6E0FEA3E0FF9001E0E0FCA3E0FD20
:107ECE00C3ED9FEC9E500222229001D3E004F022DB
:107EDE009001D3E0FFEFB406083062059001D2E4C2
:027EEE00F02280
:1095A6009001D3E0FFEF7011C2619001D47402F014
:1095B600A3E4F09001D3E004F09001D3E0FFEFB410
:1095C600011A205D179001D4E0FEA3E0FF9001C2CE
:0D95D600EEF0A3EFF0D25D9001D2E4F022A0
:109275009001D3E0FFEF7024306144C2619001D4C6
:109285007401F0A3E4F0AF567E009001D5E02FF015
:109295009001D4E03EF09001D3E004F09001D3E0DA
:1092A500FFEFB4011A205D179001D4E0FEA3E0FFA3
:1092B5009001C2EEF0A3EFF0D25D9001D2E4F0226E
:105EF6002061030260CEC2619001D3E0FFEF70160D
:105F0600AF561288EA7E009001D4EEF0A3EFF0902F
:105F160001D3E004F0229001D3E0FFEFB401389002
:105F260001D4E0FEA3E0FFEFC4F8540FC868FFEE0B
:105F3600C454F048FE9001D4EEF0A3EFF0AF561231
:105F460088EA7E009001D5E02FF09001D4E03EF083
:105F56009001D3E004F0229001D3E0FFEFB40238C1
:105F66009001D4E0FEA3E0FFEFC4F8540FC868FF29
:105F7600EEC454F048FE9001D4EEF0A3EFF0AF5615
:105F86001288EA7E009001D5E02FF09001D4E03E21
:105F9600F09001D3E004F0229001D3E0FFEFB403C8
:105FA600389001D4E0FEA3E0FFEFC4F8540FC868B0
:105FB600FFEEC454F048FE9001D4EEF0A3EFF0AF2C
:105FC600561288EA7E009001D5E02FF09001D4E0C9
:105FD6003EF09001D3E004F0229001D3E0FFEFB44D
:105FE6000416AF561288EA7E009001D6EEF0A3EFB3
:105FF600F09001D3E004F0229001D3E0FFEFB40566
:10600600389001D6E0FEA3E0FFEFC4F8540FC8684D
:10601600FFEEC454F048FE9001D6EEF0A3EFF0AFC9
:10602600561288EA7E009001D7E02FF09001D6E064
:106036003EF09001D3E004F0229001D3E0FFEFB4EC
:1060460006389001D6E0FEA3E0FFEFC4F8540FC86F
:1060560068FFEEC454F048FE9001D6EEF0A3EFF0D0
:10606600AF561288EA7E009001D7E02FF09001D655
:10607600E03EF09001D3E004F0229001D3E0FFEF80
:10608600B407459001D6E0FEA3E0FFEFC4F8540F35
:10609600C868FFEEC454F048FE9001D6EEF0A3EFB8
:1060A600F0AF561288EA7E009001D7E02FF09001FB
:1060B600D6E03EF09001DBE0FF9001D3EFF09001D7
:0960C600DAE0FF9001D2EFF022B4
:1060CF009001D3E0FFEF70279001E0E4F0A3E4F03C
:1060DF009001D6E0FEA3E0FF9001D8EEF0A3EFF021
:1060EF009001DEE4F0A3E4F09001D3E004F022206D
:1060FF0061030262A59001D3E0FFEFB4010EAF562A
:10610F001288EA8F7C9001D3E004F0229001D3E053
:10611F00FFEF6402706CE57CC454F0F57CAF56124F
:10612F0088EAEF257CF57C9001E0E0FEA3E0FF74A8
:10613F00002FF58274083EF583E57CF0AF7C7E007E
:10614F009001DFE02FF09001DEE03EF09001E1E002
:10615F0004F070069001E0E004F09001D9E024FF14
:10616F00F09001D8E034FFF09001D8E0FEA3E0FFFB
:10617F00EF4E60079001D37401F0229001D3E00439
:10618F00F0229001D3E0FFEFB40316AF561288EA66
:10619F007E009001DCEEF0A3EFF09001D3E004F06D
:1061AF00229001D3E0FFEFB404389001DCE0FEA3AE
:1061BF00E0FFEFC4F8540FC868FFEEC454F048FE78
:1061CF009001DCEEF0A3EFF0AF561288EA7E00905C
:1061DF0001DDE02FF09001DCE03EF09001D3E00410
:1061EF00F0229001D3E0FFEFB405389001DCE0FE20
:1061FF00A3E0FFEFC4F8540FC868FFEEC454F04893
:10620F00FE9001DCEEF0A3EFF0AF561288EA7E00AD
:10621F009001DDE02FF09001DCE03EF09001D3E043
:10622F0004F0229001D3E0FFEF640670699001DC67
:10623F00E0FEA3E0FFEFC4F8540FC868FFEEC454AC
:10624F00F048FE9001DCEEF0A3EFF0AF561288EAB3
:10625F007E009001DDE02FF09001DCE03EF0900138
:10626F00DCE0FEA3E0FF9001DEE0FCA3E0FDEDB576
:10627F00071AECB506169001DAE0FF9001D2EFF0A5
:10628F009001DBE0FF9001D3EFF022227F0212009A
:07629F00869001D2E4F02219
:1088EA008F7AE57AB430037F0022E57AB431037FC8
:1088FA000122E57AB432037F0222E57AB433037F98
:10890A000322E57AB434037F0422E57AB435037F7F
:10891A000522E57AB436037F0622E57AB437037F67
:10892A000722E57AB438037F0822E57AB439037F4F
:10893A000922E57AB441037F0A22E57AB442037F29
:10894A000B22E57AB443037F0C22E57AB444037F11
:10895A000D22E57AB445037F0E22E57AB446037FF9
:07896A000F22D2637F0022FF
:0B0086008F7B758400857B99D262227D
:109A3E00C2B5900003741EF0900003E0FFEF6004C7
:079A4E00C2B580F4D2B5227D
:105CF60000000000000004000000080000000C0086
:105D060000001000000014000000180000001C0035
:105D160000002000000024000000280000002C00E5
:105D260000003000000034000000380000003C0095
:105D360000004000000044000000480000004C0045
:105D460000005000000054000000580000005C00F5
:105D560000006000000064000000680000006C00A5
:105D660000007000000074000000780000007C0055
:105D760000108000001084000010880000108C00C5
:105D860000109000001094000010980000109C0075
:105D96000010A0000010A4000010A8000010AC0025
:105DA6000010B0000010B4000010B8000010BC00D5
:105DB6000010C0000010C4000010C8000010CC0085
:105DC6000010D0000010D4000010D8000010DC0035
:105DD6000010E0000010E4000010E8000010EC00E5
:105DE6000010F0000010F4000010F8000010FC0095
:105DF60000218000002184000021880000218C0001
:105E060000219000002194000021980000219C00B0
:105E16000021A0000021A4000021A8000021AC0060
:105E26000021B0000021B4000021B8000021BC0010
:105E36000021C0000021C4000021C8000021CC00C0
:105E46000021D0000021D4000021D8000021DC0070
:105E56000021E0000021E4000021E8000021EC0020
:105E66000021F0000021F4000021F8000021FC00D0
:105E760000318000003184000031880000318C0040
:105E860000319000003194000031980000319C00F0
:105E96000031A0000031A4000031A8000031AC00A0
:105EA6000031B0000031B4000031B8000031BC0050
:105EB6000031C0000031C4000031C8000031CC0000
:105EC6000031D0000031D4000031D8000031DC00B0
:105ED6000031E0000031E4000031E8000031EC0060
:105EE6000031F0000031F4000031F8000031FC0010
:104250009001ADE0FFEF70769001BFE0FFEFD394E7
:104260000340030246B42060030246B4C2609001DA
:10427000BCE51EF0A3E51FF09001BCE0FEA3E0FF4B
:10428000EE541FFE9001B6EEF0A3EFF09001BCE0FB
:10429000FEA3E0FFEEC4135407FF7E009001BCEEC6
:1042A000F0A3EFF09001BDE0FF9001AFEFF09001BF
:1042B000AEE4F09001BCE0FEA3E0FFEF4E7004D24C
:1042C0005E22229001BDE0FF9001ADEFF02290014F
:1042D000ADE0FFEFB4011A2060030246B49001B8CC
:1042E000E51EF0A3E51FF0C260D25E9001ADE4F0E0
:1042F000229001ADE0FFEF640270402060030246AF
:10430000B4C2609001AEE0FFEF70119001B8E51EFD
:10431000F0A3E51FF09001AEE004F0229001AEE0C2
:10432000FFEF640160030246B49001BAE51EF0A3FA
:10433000E51FF0D25E9001ADE4F0229001ADE0FF08
:10434000EF640360030244612060030246B49001FD
:10435000A7740AF0C2609001AEE0FFEF70299001EF
:10436000B8E51EF0A3E51FF09001B4E4F0A3E4F07B
:104370009001B0E4F0A3E4F09001B2E4F0A3E4F023
:104380009001AEE004F0229001AEE0FFEF64017016
:10439000799001BCE51EF0A3E51FF09001BCE0FEA2
:1043A000A3E0FF9001B1E02FF09001B0E03EF0906B
:1043B00001BCE0FCA3E0FD9001B2E475F0011285C0
:1043C00037AFF0FEEF25E0FFEE33FE74002FF582ED
:1043D00074043EF583ECF0A3EDF09001B5E004F039
:1043E00070069001B4E004F09001B6E0FEA3E0FF97
:1043F0009001B4E0FCA3E0FDED6F7002EC6E600391
:104400000246B49001AE7402F0229001AEE0FFEFDC
:10441000640260030246B49001BAE51EF0A3E51FF2
:10442000F09001ADE4F09001B0E0FEA3E0FF900158
:10443000BAE0FCA3E0FDEDB5071FECB5061B90014B
:10444000B6E0FEA3E0FF9001B8E0FCA3E0FD12920D
:10445000C57F007E90129A7D227F017E90129A7D08
:10446000229001ADE0FFEF640460030245922060FA
:10447000030246B49001A7740AF0C2609001AEE056
:10448000FFEF70299001B8E51EF0A3E51FF0900141
:10449000B4E4F0A3E4F09001B0E4F0A3E4F0900100
:1044A000B2E4F0A3E4F09001AEE004F0229001AE9B
:1044B000E0FFEF640170739001BCE51EF0A3E51FFF
:1044C000F09001BCE0FEA3E0FF9001B1E02FF0907E
:1044D00001B0E03EF09001BCE0FCA3E0FD9001B231
:1044E000E475F001128537AFF0FEEF25E0FFEE3303
:1044F000FE74002FF58274043EF583ECF0A3EDF01A
:104500009001B5E004F070069001B4E004F0900171
:10451000B4E0FEA3E0FFEF64007003EE640260030A
:104520000246B49001AEE004F0229001AEE0FFEF4D
:10453000640260030246B4755B559001BAE51EF053
:10454000A3E51FF09001B0E0FEA3E0FF9001BAE008
:10455000FCA3E0FDEDB50727ECB506239001B6E01E
:10456000FEA3E0FF127EF07F007E90129A7D900104
:10457000B8E0FEA3E0FFEF4E6012755CAA800D75F7
:104580005B00755C007F017E90129A7D9001ADE426
:10459000F0229001ADE0FFEF6405600302469F202A
:1045A00060030246B49001A7740AF0C2609001AEA5
:1045B000E0FFEF70299001B8E51EF0A3E51FF09031
:1045C00001B4E4F0A3E4F09001B0E4F0A3E4F090CF
:1045D00001B2E4F0A3E4F09001AEE004F022900117
:1045E000AEE0FFEF640170769001BCE51EF0A3E53C
:1045F0001FF09001BCE0FEA3E0FF9001B1E02FF0BE
:104600009001B0E03EF09001BCE0FCA3E0FD900121
:10461000B2E475F001128537AFF0FEEF25E0FFEE52
:1046200033FE74002FF58274043EF583ECF0A3EDA5
:10463000F09001B5E004F070069001B4E004F09051
:1046400001B6E0FEA3E0FF9001B4E0FCA3E0FDEDC5
:104650006F7002EC6E705D9001AEE004F02290018C
:10466000AEE0FFEF6402704C9001BAE51EF0A3E5E6
:104670001FF09001ADE4F09001B0E0FEA3E0FF90E8
:1046800001BAE0FCA3E0FDEDB5070CECB506087F30
:10469000007E90129A7D227F017E90129A7D229058
:1046A00001ADE0FFEFD39405400A9001ADE4F09036
:0546B00001AEE4F02260
:1032E8009001BFE0FFEF702A9001ADE0FFEFD394AB
:1032F80002400302384F305F0302384F205D03025B
:10330800384F9001BEE0FF9001BFEFF09001C0E49C
:10331800F0229001BFE0FFEFB401179001C2E0FE78
:10332800A3E0FFEE4420FE129A7DC25D9001BFE447
:10333800F0229001BFE0FFEF640270489001C0E006
:10334800FFEF7019205F169001C2E0FEA3E0FFEEC8
:103358004440FE129A7D9001C0E004F0229001C022
:10336800E0FFEFB4011E305F0302384F9001C4E064
:10337800FEA3E0FF129A7DC25D9001BFE4F09001C8
:10338800C0E4F0229001BFE0FFEF6403706C90018D
:10339800C0E0FFEF701C305F0302384F9001C2E0BD
:1033A800FEA3E0FFEE4460FE129A7D9001C0E004A7
:1033B800F0229001C0E0FFEFB40118305F0302383B
:1033C8004F9001C4E0FEA3E0FF129A7D9001C0E097
:1033D80004F0229001C0E0FFEFB4021E305F030248
:1033E800384F9001C6E0FEA3E0FF129A7DC25D90BF
:1033F80001BFE4F09001C0E4F0229001BFE0FFEFCC
:10340800640460030235989001C0E0FFEF703390C8
:1034180001C2E0FEA3E0FF9001C4E0FCA3E0FD12BE
:1034280091D29001CAE4F0A3E4F09001CCE4F0A3B7
:103438007480F09001C8E4F0A3E4F09001C0E004C7
:10344800F0229001C0E0FFEFB4011C305F030238A6
:103458004F9001C2E0FEA3E0FFEE4480FE129A7D89
:103468009001C0E004F0229001C0E0FFEFB4021820
:10347800305F0302384F9001C4E0FEA3E0FF129AC8
:103488007D9001C0E004F0229001C0E0FFEF6403EA
:103498007063305F0302384F9001C8E475F0011281
:1034A8008537AFF0FEEF25E0FFEE33FE74002FF511
:1034B8008274043EF583E0F570A3E0F571AF71AE58
:1034C80070129A7D9001CBE02571F09001CAE03529
:1034D80070F09001CDE024FFF09001CCE034FFF0D3
:1034E8009001CCE0FEA3E0FFEF4E600222229001A3
:1034F800C0E004F0229001C0E0FFEFB4041E305F8A
:103508000302384F9001CAE0FEA3E0FF129A7D90B3
:1035180001C17464F09001C0E004F0229001C0E0A1
:10352800FFEF6405706A9001C1E0FFEF7019900128
:10353800CFE004F070069001CEE004F09001BFE403
:10354800F09001C0E4F022306046C260851E7285AA
:103558001F739001C0E4F0E573B40011E572B490F4
:103568000C9001BFE4F09001C0E4F0C25DE5736423
:10357800017004E5726490600302384F9001C0E462
:10358800F09001CFE004F070069001CEE004F02244
:103598009001BFE0FFEF6405600302384F9001C05F
:1035A800E0FFEF702B9001CAE4F0A3E4F09001CCA7
:1035B8007402F0A3E4F09001C8E4F0A3E4F09001F1
:1035C800C2E0FEA3E0FF128B7B9001C0E004F02272
:1035D8009001C0E0FFEFB4011C305F0302384F9048
:1035E80001C2E0FEA3E0FFEE44A0FE129A7D900126
:1035F800C0E004F0229001C0E0FFEF640270633085
:103608005F0302384F9001C8E475F001128537AFA7
:10361800F0FEEF25E0FFEE33FE74002FF582740410
:103628003EF583E0F570A3E0F571AF71AE70129AC4
:103638007D9001CBE02571F09001CAE03570F090E3
:1036480001CDE024FFF09001CCE034FFF09001CCF4
:10365800E0FEA3E0FFEF4E600222229001C0E004EA
:10366800F0229001C0E0FFEFB4031E305F03023880
:103678004F9001CAE0FEA3E0FF129A7D9001C17449
:1036880064F09001C0E004F0229001C0E0FFEF6414
:103698000470659001C1E0FFEF70149001CFE00461
:1036A800F070069001CEE004F09001C0E4F0223002
:1036B8006046C260851E72851F739001C0E4F0E504
:1036C80073B40011E572B4900C9001BFE4F090015E
:1036D800C0E4F0C25DE57364017004E57264906053
:1036E8000302384F9001CFE004F070069001CEE05D
:1036F80004F09001C0E4F0229001C0E0FFEF7020D8
:103708009001CAE4F0A3E4F09001CC7402F0A3E4C1
:10371800F09001C8E4F0A3E4F09001C0E004F022C6
:103728009001C0E0FFEFB4011C305F0302384F90F6
:1037380001C2E0FEA3E0FFEE44C0FE129A7D9001B4
:10374800C0E004F0229001C0E0FFEF640270633033
:103758005F0302384F9001C8E475F001128537AF56
:10376800F0FEEF25E0FFEE33FE74002FF5827404BF
:103778003EF583E0F570A3E0F571AF71AE70129A73
:103788007D9001CBE02571F09001CAE03570F09092
:1037980001CDE024FFF09001CCE034FFF09001CCA3
:1037A800E0FEA3E0FFEF4E600222229001C0E00499
:1037B800F0229001C0E0FFEFB4031E305F0302382F
:1037C8004F9001CAE0FEA3E0FF129A7D9001C0E08D
:1037D80004F09001C17464F0229001C0E0FFEF642E
:1037E8000470649001C1E0FFEF70199001CFE0040C
:1037F800F070069001CEE004F09001C0E4F0900172
:10380800BFE4F022306040C260851E72851F73904D
:1038180001C0E4F0E573B40011E572B4900C9001B6
:10382800BFE4F09001C0E4F0C25DE573B40118E5AF
:1038380072B490139001C0E4F09001CFE004F070EE
:07384800069001CEE004F040
:01384F002256
:047EF0008E0F8F1052
:107EF400D3E510947DE50F940040047F0180027F58
:107F040000C3E510943FE50F940050047E01800205
:107F14007E00EE4FFFEF6003027FECE510AE0F78BA
:107F240002C333CE33CED8F9FF74F82FF582745CD4
:107F34003EF583E493F511740193F512E510AE0F49
:107F44007802C333CE33CED8F9FF74F62FF582749A
:107F54005C3EF583E493FE740193FF8F179001ADAB
:107F6400E0FFEF6405FF9001E8EFF09001AEE0FF61
:107F7400EF6401FF9001E9EFF0AD12AC11AF1712FD
:107F840095699001ADE0FFEF6405FF9001E8EFF023
:107F94009001AEE0FFEF6403FF9001E9EFF0751587
:107FA40000751600C3E51594045033AE15AF16746E
:107FB400002FF58274043EF583E0FF7E008E138F5C
:107FC40014AB14AD12AC11AF1712939B0512E5124A
:107FD400700205110516E5167002051580C690019C
:087FE400E8E4F09001E9E4F08B
:017FEC002272
:0892C5008E648F658C668D67D5
:1092CD00756800756900E56525E0FFE56433FEC34B
:1092DD00E5699FE5689E50290567E567AE667002F2
:1092ED00056614FFAC68AD6974002DF58274043CFD
:1092FD00F583E0FD1273760569E5697002056880F6
:01930D00C59A
:01930E00223C
:048B7B008E5D8F5E1E
:108B7F00E55EAE5D7802C333CE33CED8F9FF74F81D
:108B8F002FF582745C3EF583E493F55F740193F5E2
:108B9F0060E55EAE5D7802C333CE33CED8F9FF7495
:108BAF00F62FF582745C3EF583E493FE740193FF18
:108BBF008F63756100756200C3E5619404502BAD3E
:108BCF0060AC5FAF6312995CAC61AD6274002DF560
:108BDF008274043CF583EFF00560E5607002055F79
:0A8BEF000562E5627002056180CEA8
:018BF9002259
:0891D2008E6A8F6B8C6C8D6DB1
:1091DA00756E00756F00E56B2401FFE56A3400FEC9
:1091EA00EF25E0FFEE33FEC3E56F9FE56E9E502943
:1091FA00056DE56DAE6C7002056C14FF1273B7ACA9
:10920A006EAD6F74002DF58274043CF583EFF005A2
:09921A006FE56F7002056E80BD66
:019223002228
:109A7D008E188F19205FFD851825851926755A00BA
:039A8D00D25F2283
:1075EF00205E030277299001AFE0FFEF6003027680
:1075FF00B6C25E9001B6E0FEA3E0FFEFB4FF0BEE64
:10760F00B41F0775840075EF03229001B6E0FEA347
:10761F00E0FFEEFF7E008F789001B7E0FFEF54FFA1
:10762F00F579E578700B7FFF8F799001E57401F0A4
:10763F0022E578B41516C3E579648094B3500D90A4
:10764F0001E27401F09001E4E579F022E578B416D7
:10765F0016C3E579648094F2500D9001E27402F044
:10766F009001E4E579F022D3E57864809480403787
:10767F00C3E57864809495502ED3E5796480948027
:10768F004025AF79EF3395E0FEC3EF94FBEE6480B6
:10769F00948050139001E27403F09001E3E578F0C9
:1076AF009001E4E579F0229001AFE0FFEF64027002
:1076BF00699001B6E0FEA3E0FFEF64014E702B90DE
:1076CF0001BFE0FFEF70F89001C2E4F0A3747FF008
:1076DF009001BAE0FEA3E0FF9001C4EEF0A3EFF03B
:1076EF009001BE7404F0D25DC25E9001B6E0FEA3BD
:1076FF00E0FFEF64024E70229001BFE0FFEF70F8E1
:10770F009001BAE0FEA3E0FF9001C2EEF0A3EFF00C
:0A771F009001BE7405F0D25DC25E59
:01772900223D
:10FC0000C2AF12FCD812FD10E4F550F551E42551B5
:10FC1000FFE5503480FE12FCB6AD07AF51AE501276
:10FC2000FC5F0551E55170020550C3E550948040DA
:10FC3000DC755080755100AF51AE5012FCC7AD0756
:10FC4000AF51AE5012FC8A0551E55170020550C308
:10FC5000E55094F440E1D2AF75840075EF0122C203
:10FC6000AF75840F53A1FEE4F5B1F58443B701F5F8
:10FC700084438F018E088F098F828E83EDF0E4F527
:10FC800084538FFEF58453B7FE22C2AF75840F53A1
:10FC9000A1FE75B110E4F58443B701F584438F01EB
:10FCA0008E088F098F828E83EDF0E4F584538FFEEA
:10FCB000F58453B7FE22C2AF75B1218E0A8F0B8F28
:10FCC000828E83E493FF22C2AF75B1318E0A8F0B0F
:10FCD0008F828E83E493FF22C2AFE4FFFEE4F5B18E
:10FCE000F58443B701F584758F03AD07AC068C0826
:10FCF0008D098D828C83F0F58FF58453B7FE2FFF2D
:10FD000074043EFEC3948040D4E4F58453B7FE22CD
:10FD1000C2AF7F007E8075B110E4F58443B701F572
:04FD200084758F0354
:10FD2400AD07AC068C088D098D828C83F0F58FF5B8
:10FD34008453B7FE2FFF74043EFEC3648094744062
:08FD4400D1E4F58453B7FE225F
:0300000002007685
:0C007600787FE4F6D8FD7581A20262A636
:1084CD00BB010689828A83E0225002E722BBFE02AD
:0984DD00E32289828A83E49322E0
:1084E600BB010CE58229F582E5833AF583E022504B
:1084F60006E92582F8E622BBFE06E92582F8E22295
:0D850600E58229F582E5833AF583E49322AE
:10851300BB010689828A83F0225002F722BBFE0147
:02852300F32241
:10852500EF8DF0A4A8F0CF8CF0A428CE8DF0A42E6A
:02853500FE2224
:10853700A3F8E0C5F025F0F0E582158270021583F7
:06854700E0C838F0E82254
:10854D00D083D082F8E4937012740193700DA3A3BD
:10855D0093F8740193F5828883E4737402936860D1
:06856D00EFA3A3A380DFD1
:00000001FF
